:020000040000FA
:06000000DDEF3DF01200EF
:06080000DDEF3DF01200E7
:06082A000600927C0000B4
:10083000E90100000C000000917C0000B5020000FE
:10084000010000008B7C0000FA00000006000000A0
:10085000137C0000B4020000010000007E7C000058
:10086000DC0100000D0000007A7C0000AA020000FC
:040870000400000080
:0C08740004001200D9CFE6FFE1CFD9FF4D
:1008800081E945E8030E056E0101E551010A17E013
:10089000010A2AE10A0EE45D09E10001DA51016E64
:1008A000DB51026EDC51036EDD511DD0020100519F
:1008B000016E0151026E0251036E035114D00A0EF3
:1008C000E45D09E10001DE51016EDF51026EE0518D
:1008D000036EE15108D002010451016E0551026E10
:1008E0000651036E0751046E90EC0AF0030A2DE0E6
:1008F000070A1BE0010A0AE0050A04E0010A02E017
:10090000030A35E17A0EE66E730E34D0750EE66E8C
:10091000730E06EC0AF00001CB51E66EE66A030E98
:10092000E66ECF0EE66E000E2CD0700EE66E730EE5
:1009300006EC0AF0DCC1E6FFDDC1E6FFDEC1E6FF42
:10094000DFC1E6FF94EC0AF017D06B0EE66E730E73
:1009500006EC0AF0E0C1E6FFE1C1E6FFE2C1E6FF16
:10096000E3C1E6FF94EC0AF0040E056E05D0660EB6
:10097000E66E730E06EC0AF00101E55106E159EC52
:100980000AF0E66E2DEC36F005D059EC0AF0E66E72
:1009900066EC36F045E946E9E7CFD9FF1200D9CF3A
:1009A000E6FFE1CFD9FF81E958E8136A146A156AB6
:1009B000166A176A186AF70E926ED00E936E380E8A
:1009C000946EF19E8A86D0B604D0E66AD0EC2EF002
:1009D00041E9170EE66ED7EC3CF041E952EC0AF023
:1009E000750EE66E9CEC3CF041E989EC0AF00101E1
:1009F000E451FF0A02E175EF09F0F40A01E16AD35C
:100A0000010A01E1C4D2030A01E12DD2010A01E188
:100A100017D20F0A01E1FED1010A01E1D5D1030A83
:100A200001E1BFD1010A01E1AAD1070A01E1A2D186
:100A3000010A01E196D1030A01E187D1010A02E02E
:100A400083EF09F0D60EF66E750EF76E0900F5CF3E
:100A500060F00900F5CF61F00900F5CF62F0090000
:100A6000F5CF63F00900F5CF64F00900F5CF65F02C
:100A70000900F5CF66F00900F5CF67F00900F5CF62
:100A800068F00900F5CF69F00900F5CF6AF00900B8
:100A9000F5CF6BF00900F5CF6CF00900F5CF6DF0E4
:100AA0000900F5CF6EF00900F5CF6FF00900F5CF22
:100AB00070F00900F5CF71F00900F5CF72F0090070
:100AC000F5CF73F00900F5CF74F00900F5CF75F09C
:100AD0000900F5CF76F00900F5CF77F00900F5CFE2
:100AE00078F00900F5CF79F00900F5CF7AF0090028
:100AF000F5CF7BF00900F5CF7CF00900F5CF7DF054
:100B00000900F5CF7EF00900F5CF7FF00900F5CFA1
:100B100080F00900F5CF81F00900F5CF82F00900DF
:100B2000F5CF83F00900F5CF84F00900F5CF85F00B
:100B30000900F5CF86F00900F5CF87F00900F5CF61
:100B400088F00900F5CF89F00900F5CF8AF0090097
:100B5000F5CF8BF00900F5CF8CF00900F5CF8DF0C3
:100B60000900F5CF8EF00900F5CF8FF00900F5CF21
:100B700090F00900F5CF91F00900F5CF92F009004F
:100B8000F5CF93F00900F5CF94F00900F5CF95F07B
:100B90000900F5CF96F00900F5CF97F00900F5CFE1
:100BA00098F00900F5CF99F00900F5CF9AF0090007
:100BB000F5CF9BF00900F5CF9CF00900F5CF9DF033
:100BC0000900F5CF9EF00900F5CF9FF00900F5CFA1
:100BD000A0F00900F5CFA1F00900F5CFA2F00900BF
:100BE000F5CFA3F00900F5CFA4F00900F5CFA5F0EB
:100BF0000900F5CFA6F00900F5CFA7F00900F5CF61
:100C0000A8F00900F5CFA9F00900F5CFAAF0090076
:100C1000F5CFABF00900F5CFACF00900F5CFADF0A2
:100C20000900F5CFAEF00900F5CFAFF00900F5CF20
:100C3000B0F00900F5CFB1F00900F5CFB2F009002E
:100C4000F5CFB3F00900F5CFB4F00900F5CFB5F05A
:100C50000900F5CFB6F00900F5CFB7F00900F5CFE0
:100C6000B8F00900F5CFB9F00900F5CFBAF00900E6
:100C7000F5CFBBF00900F5CFBCF00900F5CFBDF012
:100C80000900F5CFBEF00900F5CFBFF00900F5CFA0
:100C9000C0F00900F5CFC1F00900F5CFC2F009009E
:100CA000F5CFC3F00900F5CFC4F00900F5CFC5F0CA
:100CB0000900F5CFC6F00800F5CFC7F00001C7B7AF
:100CC0001CD02F0EC16F400EC06FC26FC787C79177
:100CD000C783C7953C0EC36FC46B0F0EC56FC66B41
:100CE000C789C78DC79BC78F600EE66E000EE66E84
:100CF00001EC24F042E9680EBFDBECEC20F0ADEC37
:100D00002DF05BEC29F0EDEC11F0DCEC1CF03D0E6D
:100D1000F66E760EF76E0800F550080B02E1BDEC9A
:100D20002DF05CEC2EF0380E946EAAEC21F081A828
:100D300084D00001C7A907D00101010EE46F0001B2
:100D4000C96BCA6BE0D2CDDBDED20001C8B303D0E1
:100D50000101020EE46F020E0101E55D01E0D3D254
:100D600031D00001C8B3BDDB020E0101E55D01E039
:100D7000CAD228D0BEDBC8A1C6D2010123D0E1DB94
:100D8000CCBFCD69B3EC0AF09EDB0001C8A102D054
:100D90000101E4690101CB5101E1B5D20101050E68
:100DA000B1D2C0C0C9F0C1C0CAF05C0EE66E730E0D
:100DB0002DDB0101CB5102E101019BDB0001C8A148
:100DC000A2D20101E4699FD2E551020A15E0030AAB
:100DD00007E0010A1BE1B5DBCCBFCD69C4DB0AD05B
:100DE000570EE66E730E12DB02EC2EF0F3CFE6FF29
:100DF000F4CFE6FF68DB0AD0E56B0001C8A306D09C
:100E0000C9693F0ECA6F0101010EE86F0001C8B346
:100E10007AD276D2E551020A06E0020A02E0010A1D
:100E200003E12ADD01D0E56B0001C8A303D0010175
:100E3000080EE46F0001C8B166D20101030E62D250
:100E40007D0EE66E7CEC3CF041E9000EE66EE66A53
:100E500026EC3DF042E90101E56B24DB156A166AD8
:100E60000101090EE46F5CDB000A1EE0010A18E0D4
:100E7000030A12E0010A0CE0070A06E0010A18E181
:100E8000520EE66E730E13D04D0EE66E730E0FD03B
:100E9000480EE66E730E0BD0430EE66E730E07D04F
:100EA0003E0EE66E730E03D0390EE66E730EAEDAAA
:100EB0000001C8B302D00101E4693EEC3DF00ADB59
:100EC00001E321D23EEC3DF0E5DA26EC3DF042E9CB
:100ED000152A000E1622020EE66EE66AC5C0E6FF6F
:100EE000C6C0E6FFA8EC2CF0FE0EE350155C41E90D
:100EF000E550165801E207D200C2DAF001C2DBF079
:100F000002C2DCF003C2DDF004C2DEF005C2DFF095
:100F100006C2E0F007C2E1F00101E56B01010351F7
:100F2000056E0451066E0551076E0651086E075195
:100F3000096E08510A6E09510B6E0A510C6E0B5165
:100F40000D6E0C510E6E0D510F6E0E51106EE66A45
:100F500030EC2AF041E9116A126AD890125004E686
:100F60005E0E115C010E125802E25ADAF6D7C9C0C1
:100F7000E6FF30EC2AF041E92EEC3EF001010A0ECA
:100F8000E46F02014651176E4751186EBCD1E5510E
:100F9000030A31E0010A06E0020A02E0010A2CE13C
:100FA0006BDC2AD0BDDA000A14E01750E708030E04
:100FB000185412E2340EE66E730E28DA0101E80EC0
:100FC000175CCC6F030E1858CD6FCCC1E6FFE66EF0
:100FD0000BD00101E56B10D02F0EE66E730E16DA02
:100FE00017EBE6FF18EBE6FF030EE66ECF0EE66E9C
:100FF000000EBEDA01D0E56B020E0001C8155DE1FE
:101000000101E7515AE18CDA010A49E0030A3EE0A6
:10101000010A38E0070A32E0010A45E1CB510C0D24
:1010200002018851F324E96E8951F420EA6E05EB40
:10103000EEFF06EBEEFF07EBEEFF08EBEEFF09EB32
:10104000EEFF0AEBEEFF0BEBEEFF0CEBEEFF0DEB12
:10105000EEFF0EEBEEFF0FEBEEFF10EBEEFF0001ED
:10106000CB2B380ECB5D1FE301010B0EE46F0001AB
:10107000CB6BCC6BD5EC25F06DDA15D0ECD93CEC14
:101080001FF010D0E8D9F7EC1EF00CD0D950050FA6
:10109000E66EDACFE6FF51EC1FF042E904D0DBD96F
:1010A0005CEC1EF048E90001C7AD04D00101010E5F
:1010B000E76F03D00101070EE46F020E0001C815AF
:1010C00001E121D10101E75101E11DD1080EE46FD9
:1010D000E76B19D10001CC51010BE66EE9EC25F06C
:1010E00041E9AED90001CC2B2A0EE66E730E8ED9E3
:1010F0000001CC51E66EE66A020EE66ED00EE66E98
:10110000000E36DA640E0001CC5D01E0FCD0A0C711
:1011100060F0A1C761F0A2C762F0A3C763F0A4C7E3
:1011200064F0A5C765F0A6C766F0A7C767F0A8C7B3
:1011300068F0A9C769F0AAC76AF0ABC76BF0ACC783
:101140006CF0ADC76DF0AEC76EF0AFC76FF0B0C753
:1011500070F0B1C771F0B2C772F0B3C773F0B4C723
:1011600074F0B5C775F0B6C776F0B7C777F0B8C7F3
:1011700078F0B9C779F0BAC77AF0BBC77BF0BCC7C3
:101180007CF0BDC77DF0BEC77EF0BFC77FF0C0C793
:1011900080F0C1C781F0C2C782F0C3C783F0C4C763
:1011A00084F0C5C785F0C6C786F0C7C787F0C8C733
:1011B00088F0C9C789F0CAC78AF0CBC78BF0CCC703
:1011C0008CF0CDC78DF0CEC78EF0CFC78FF0D0C7D3
:1011D00090F0D1C791F0D2C792F0D3C793F0D4C7A3
:1011E00094F0D5C795F0D6C796F0D7C797F0D8C773
:1011F00098F0D9C799F0DAC79AF0DBC79BF0DCC743
:101200009CF0DDC79DF0DEC79EF0DFC79FF0E0C712
:10121000A0F0E1C7A1F0E2C7A2F0E3C7A3F0E4C7E2
:10122000A4F0E5C7A5F0E6C7A6F0E7C7A7F0E8C7B2
:10123000A8F0E9C7A9F0EAC7AAF0EBC7ABF0ECC782
:10124000ACF0EDC7ADF0EEC7AEF0EFC7AFF0F0C752
:10125000B0F0F1C7B1F0F2C7B2F0F3C7B3F0F4C722
:10126000B4F0F5C7B5F0F6C7B6F0F7C7B7F0F8C7F2
:10127000B8F0F9C7B9F0FAC7BAF0FBC7BBF0FCC7C2
:10128000BCF0FDC7BDF0FEC7BEF0FFC7BFF0CD513B
:10129000070BF36EF80EC715F310C76F600EECD88E
:1012A000116A126A640ED89012BE03D0115C000E4F
:1012B000125802E2B5D8F6D724D9640ED89012BEDF
:1012C00003D0115C000E125802E2AAD8F6D719D941
:1012D000640ED89012BE03D0115C000E125802E2C8
:1012E0009FD8F6D701010A0E0DD0E8C1E6FFD0EC79
:1012F0002EF041E915D9CD6FC781C793C785CB6B58
:101300000101070EE46FC0EC15F00001C86B8150BD
:10131000100B01E0010EC82754EC2EF0000906E086
:10132000020E0001C827F5D8136A146AC0EC15F044
:101330003AEC04F0B5EC21F0C0EC15F0040E01011C
:10134000E76E661902E7663502D06651E75C12E285
:10135000250EE66E730E5AD8E66A650EE66E010E2D
:10136000E66E010EE66ED00EE66E000EE66E8BECBB
:1013700036F046E9CE0EE66E000EE66E97EC2AF0E9
:1013800042E99EEC3DF0F9D80001C2510101CF6B5A
:10139000C2C0CFF1CE6BF350CE5DF450CF5905E211
:1013A0000101E52B5CEC2EF07DD8C0EC15F06EEC65
:1013B0003DF090D822E26EEC3DF06CD856EC3DF05A
:1013C00042E9132A000E14220001C351C41115E092
:1013D000140EE66EE66AC3C0E6FFC4C0E6FFA8ECE2
:1013E0002CF0FE0EE350D8801354145041E9E55818
:1013F00004E2E66AD0EC2EF041E9C0EC15F0C9C079
:10140000E6FF30EC2AF041E9F7EF04F0E66EE66A19
:10141000CE0EE66E000EE66E5DEC34F045E912008D
:101420008A84990EE66EF6EC3DF041E98A94990EB5
:10143000E66EF6EC3DF041E9112A000E1222120090
:1014400089D80101CC51016ECD51026ECE51036E8F
:10145000CF51046E1200DEC0E6FFDFC0E6FFE0C041
:10146000E6FFE1C0E6FFDAC0E6FFDBC0E6FFDCC076
:10147000E6FFDDC0E6FF1200E66EE66A600EE66E8D
:10148000000EE66ED60EE66E750EE66E9EEC1DF054
:1014900046E9120072D80101A80ECC5F610ECD5B47
:1014A000B3EF0AF0000EE66EE66A86EC3DF042E924
:1014B000120003EBE6FF04EBE6FF05EBE6FFCE0EC2
:1014C000E66E000E1200030EE66ECE0EE66E000E05
:1014D000B8EF0AF052D80101F350A808610EF45495
:1014E00012000101060EE46FC0C0C9F0C1C0CAF00D
:1014F0001200040EE46F0001010EC96F110ECA6FD5
:1015000012001E0EE66EBCEC3CF041E9116A126A54
:101510001200000EE66EE66A56EC3DF042E912005B
:101520000001C751070B120001EBE6FF02EBE6FFDB
:1015300003EBE6FF04EBE6FFDDEC34F048E920EFD7
:101540000AF0610EE66E730E61DFA1C2CCF10101FB
:10155000CD6B1200A2C2CCF1A3C2CDF1A4C2CEF1D8
:10156000A5C2CFF11200CCC1E6FFCDC1E6FF12004B
:10157000E66E2DEC36F045E91200F3CFCCF1F4CF56
:04158000CDF1120097
:0C15840003EBE6FF04EBE6FF05EBE6FFDF
:1015900006EBE6FFEECFE6FFEECFE6FFEECFE6FF8F
:1015A000EECFE6FFE9EC34F007EBE6FF08EBE6FFF1
:1015B00009EBE6FF0AEBE6FF08E8EECFE6FFEECF29
:1015C000E6FFEECFE6FFEECFE6FFE9EC34F02D507C
:1015D00029262E502A222F502B2230502C2244E92B
:1015E0000BEBE6FF0CEBE6FF0DEBE6FF0EEBE6FF89
:1015F00008E8EECFE6FFEECFE6FFEECFE6FFEECF58
:10160000E6FFE9EC34F02D5029262E502A222F50E7
:101610002B2230502C2244E908E8EECFE6FFEECF33
:10162000E6FFEECFE6FFEECFE6FF2D5029262E5047
:101630002A222F502B2230502C2244E924E903EB9C
:10164000E6FF04EBE6FF05EBE6FF06EBE6FFEECF79
:10165000E6FFEECFE6FFEECFE6FFEECFE6FFE9ECEA
:1016600034F007EBE6FF08EBE6FF09EBE6FF0AEBD9
:10167000E6FF08E8EECFE6FFEECFE6FFEECFE6FFAF
:10168000EECFE6FFE9EC34F031502D2632502E2219
:1016900033502F223450302244E90BEBE6FF0CEBA1
:1016A000E6FF0DEBE6FF0EEBE6FF08E8EECFE6FF08
:1016B000EECFE6FFEECFE6FFEECFE6FFE9EC34F04B
:1016C00031502D2632502E2233502F2234503022CA
:1016D00044E908E8EECFE6FFEECFE6FFEECFE6FF07
:1016E000EECFE6FF31502D2632502E2233502F22DE
:1016F0003450302244E924E903EBE6FF04EBE6FF33
:1017000005EBE6FF06EBE6FFEECFE6FFEECFE6FFEA
:10171000EECFE6FFEECFE6FFE9EC34F007EBE6FFB5
:1017200008EBE6FF09EBE6FF0AEBE6FF08E8EECF81
:10173000E6FFEECFE6FFEECFE6FFEECFE6FFE9EC09
:1017400034F035503126365032223750332238505B
:10175000342244E90BEBE6FF0CEBE6FF0DEBE6FF72
:101760000EEBE6FF08E8EECFE6FFEECFE6FFEECFAA
:10177000E6FFEECFE6FFE9EC34F035503126365087
:101780003222375033223850342244E908E8EECF71
:10179000E6FFEECFE6FFEECFE6FFEECFE6FF3550F9
:1017A000312636503222375033223850342244E921
:1017B00024E9E552E5500E6EE5500D6EE5500C6ED5
:1017C000E7500B6EE552E5500A6EE550096EE550A4
:1017D000086EE750076EE552E550066EE550056E5F
:1017E000E550046EE750036E000CD89006BED8801A
:1017F000063205320432D8900ABED8800A32093245
:101800000832D8900EBED8800E320D320C32000C49
:10181000036A046AEE50056EEE50066E076A086AA7
:10182000EE50096EEE500A6E0B6A0C6AEE500D6EA9
:10183000EE500E6E000C64E8D9CFE6FFDACFE6FF7B
:10184000E1CFD9FFE2CFDAFFA9E901EBE9FF02EB33
:10185000EAFF06E8DDDFC9DFC8DF00EE60F092DEF8
:1018600083EB0FF084EB10F085EB11F086EB12F0B8
:1018700087EB13F088EB14F089EB15F08AEB16F088
:101880008BEB17F08CEB18F08DEB19F08EEB1AF058
:1018900001EBE9FF02EBEAFFBBDFA7DFA6DFA5DF75
:1018A00000EE90F06FDE03EBE6FF04EBE6FF05EBE6
:1018B000E6FF06EBE6FF03EBE6FF04EBE6FF05EBD6
:1018C000E6FF06EBE6FFE9EC34F007EBE6FF08EB9A
:1018D000E6FF09EBE6FF0AEBE6FF07EBE6FF08EBA6
:1018E000E6FF09EBE6FF0AEBE6FFE9EC34F00BEB71
:1018F000E6FF0CEBE6FF0DEBE6FF0EEBE6FF0BEB76
:10190000E6FF0CEBE6FF0DEBE6FF0EEBE6FFE9EC86
:1019100034F031502D2632502E2233502F223450A5
:10192000302244E92D5029262E502A222F502B22D6
:1019300030502C2244E90201295038272A503923FB
:101940002B503A232C503B23FC0EE3CFE6FFE3CF92
:10195000E6FFE3CFE6FFE3CFE6FF94EC35F0FC0EC5
:10196000E3CFE6FFE3CFE6FFE3CFE6FFE3CFE6FF1B
:1019700003EBE6FF04EBE6FF05EBE6FF06EBE6FF15
:10198000E9EC34F0E552E550066EE550056EE550A1
:10199000046EE750036EFC0EE3CFE6FFE3CFE6FFF5
:1019A000E3CFE6FFE3CFE6FF07EBE6FF08EBE6FF5A
:1019B00009EBE6FF0AEBE6FFE9EC34F0E552E5500F
:1019C0000A6EE550096EE550086EE750076EFC0E92
:1019D000E3CFE6FFE3CFE6FFE3CFE6FFE3CFE6FFAB
:1019E0000BEBE6FF0CEBE6FF0DEBE6FF0EEBE6FF85
:1019F000E9EC34F0E552E5500E6EE5500D6EE55021
:101A00000C6EE7500B6EE9EC34F0020129502027F0
:101A10002A5021232B5022232C50232344E90FEB5F
:101A2000E6FF10EBE6FF11EBE6FF12EBE6FF0FEB34
:101A3000E6FF10EBE6FF11EBE6FF12EBE6FFE9EC49
:101A400034F013EBE6FF14EBE6FF15EBE6FF16EBC5
:101A5000E6FF13EBE6FF14EBE6FF15EBE6FF16EBF4
:101A6000E6FFE9EC34F017EBE6FF18EBE6FF19EBC5
:101A7000E6FF1AEBE6FF17EBE6FF18EBE6FF19EBC4
:101A8000E6FF1AEBE6FFE9EC34F031502D26325038
:101A90002E2233502F223450302244E92D50292653
:101AA0002E502A222F502B2230502C2244E90201A2
:101AB00029503C272A503D232B503E232C503F23B6
:101AC000FC0EE3CFE6FFE3CFE6FFE3CFE6FFE3CF95
:101AD000E6FF94EC35F0FC0EE3CFE6FFE3CFE6FF44
:101AE000E3CFE6FFE3CFE6FF0FEBE6FF10EBE6FF09
:101AF00011EBE6FF12EBE6FFE9EC34F0E552E550BE
:101B0000126EE550116EE550106EE7500F6EFC0E30
:101B1000E3CFE6FFE3CFE6FFE3CFE6FFE3CFE6FF69
:101B200013EBE6FF14EBE6FF15EBE6FF16EBE6FF23
:101B3000E9EC34F0E552E550166EE550156EE550CF
:101B4000146EE750136EFC0EE3CFE6FFE3CFE6FF23
:101B5000E3CFE6FFE3CFE6FF17EBE6FF18EBE6FF88
:101B600019EBE6FF1AEBE6FFE9EC34F0E552E5503D
:101B70001A6EE550196EE550186EE750176EE9ECD5
:101B800034F00201295024272A5025232B502623E4
:101B90002C50272344E907EBE6FF08EBE6FF09EBAF
:101BA000E6FF0AEBE6FF17EBE6FF18EBE6FF19EBA3
:101BB000E6FF1AEBE6FFE9EC34F00BEBE6FF0CEB8B
:101BC000E6FF0DEBE6FF0EEBE6FF13EBE6FF14EB93
:101BD000E6FF15EBE6FF16EBE6FFE9EC34F02D50DF
:101BE000295E2E502A5A2F502B5A30502C5A44E935
:101BF0000BEBE6FF0CEBE6FF0DEBE6FF0EEBE6FF73
:101C00000FEBE6FF10EBE6FF11EBE6FF12EBE6FF52
:101C1000E9EC34F003EBE6FF04EBE6FF05EBE6FF4F
:101C200006EBE6FF17EBE6FF18EBE6FF19EBE6FF26
:101C30001AEBE6FFE9EC34F031502D5E32502E5AAB
:101C400033502F5A3450305A44E903EBE6FF04EB8B
:101C5000E6FF05EBE6FF06EBE6FF13EBE6FF14EB12
:101C6000E6FF15EBE6FF16EBE6FFE9EC34F007EBD9
:101C7000E6FF08EBE6FF09EBE6FF0AEBE6FF0FEBFA
:101C8000E6FF10EBE6FF11EBE6FF12EBE6FFE9ECF7
:101C900034F03550315E3650325A3750335A38505E
:101CA000345A44E9E552E5501A6EE550196EE55094
:101CB000186EE750176EE552E550166EE550156E3A
:101CC000E550146EE750136EE552E550126EE55084
:101CD000116EE550106EE7500F6E0FEBE6FF10EB44
:101CE000E6FF11EBE6FF12EBE6FF0FEBE6FF10EB72
:101CF000E6FF11EBE6FF12EBE6FFE9EC34F013EB45
:101D0000E6FF14EBE6FF15EBE6FF16EBE6FF13EB41
:101D1000E6FF14EBE6FF15EBE6FF16EBE6FFE9EC5A
:101D200034F017EBE6FF18EBE6FF19EBE6FF1AEBD2
:101D3000E6FF17EBE6FF18EBE6FF19EBE6FF1AEB01
:101D4000E6FFE9EC34F031502D2632502E2233508C
:101D50002F223450302244E92D5029262E502A2299
:101D60002F502B2230502C2244E9020129504027C9
:101D70002A5041232B5042232C504323FC0EE3CF07
:101D8000E6FFE3CFE6FFE3CFE6FFE3CFE6FF94EC29
:101D900035F0FC0EE3CFE6FFE3CFE6FFE3CFE6FF4F
:101DA000E3CFE6FF0FEBE6FF10EBE6FF11EBE6FFFC
:101DB00012EBE6FFE9EC34F0E552E550126EE55027
:101DC000116EE550106EE7500F6EFC0EE3CFE6FF8C
:101DD000E3CFE6FFE3CFE6FFE3CFE6FF13EBE6FF5B
:101DE00014EBE6FF15EBE6FF16EBE6FFE9EC34F04B
:101DF000E552E550166EE550156EE550146EE7504D
:101E0000136EFC0EE3CFE6FFE3CFE6FFE3CFE6FF82
:101E1000E3CFE6FF17EBE6FF18EBE6FF19EBE6FF73
:101E20001AEBE6FFE9EC34F0E552E5501A6EE550A6
:101E3000196EE550186EE750176EE9EC34F00201A8
:101E4000295028272A5029232B502A232C502B2372
:101E500044E9100E0060B4D113EBE6FF14EBE6FF8B
:101E600015EBE6FF16EBE6FF0BEBE6FF0CEBE6FFF0
:101E70000DEBE6FF0EEBE6FFE9EC34F017EBE6FFC7
:101E800018EBE6FF19EBE6FF1AEBE6FF07EBE6FFC0
:101E900008EBE6FF09EBE6FF0AEBE6FFE9EC34F0BE
:101EA0002D50295E2E502A5A2F502B5A30502C5A22
:101EB00044E917EBE6FF18EBE6FF19EBE6FF1AEB38
:101EC000E6FF03EBE6FF04EBE6FF05EBE6FF06EBC0
:101ED000E6FFE9EC34F00FEBE6FF10EBE6FF11EB69
:101EE000E6FF12EBE6FF0BEBE6FF0CEBE6FF0DEB7C
:101EF000E6FF0EEBE6FFE9EC34F031502D5E325098
:101F00002E5A33502F5A3450305A44E90FEBE6FF23
:101F100010EBE6FF11EBE6FF12EBE6FF07EBE6FF47
:101F200008EBE6FF09EBE6FF0AEBE6FFE9EC34F02D
:101F300013EBE6FF14EBE6FF15EBE6FF16EBE6FF0F
:101F400003EBE6FF04EBE6FF05EBE6FF06EBE6FF3F
:101F5000E9EC34F03550315E3650325A3750335A4E
:101F60003850345A44E9E552E550266EE550256E66
:101F7000E550246EE750236EE552E550226EE550A1
:101F8000216EE550206EE7501F6EE552E5501E6E43
:101F9000E5501D6EE5501C6EE7501B6E1BEBE6FF17
:101FA0001CEBE6FF1DEBE6FF1EEBE6FF1BEBE6FF7F
:101FB0001CEBE6FF1DEBE6FF1EEBE6FFE9EC34F061
:101FC0001FEBE6FF20EBE6FF21EBE6FF22EBE6FF4F
:101FD0001FEBE6FF20EBE6FF21EBE6FF22EBE6FF3F
:101FE000E9EC34F023EBE6FF24EBE6FF25EBE6FF1C
:101FF00026EBE6FF23EBE6FF24EBE6FF25EBE6FF0F
:1020000026EBE6FFE9EC34F031502D2632502E223B
:1020100033502F223450302244E92D5029262E509F
:102020002A222F502B2230502C2244E994EC35F0F8
:10203000FC0EE3CFE6FFE3CFE6FFE3CFE6FFE3CF1F
:10204000E6FF1BEBE6FF1CEBE6FF1DEBE6FF1EEBDE
:10205000E6FFE9EC34F0E552E5501E6EE5501D6EEA
:10206000E5501C6EE7501B6EFC0EE3CFE6FFE3CF9E
:10207000E6FFE3CFE6FFE3CFE6FF1FEBE6FF20EB53
:10208000E6FF21EBE6FF22EBE6FFE9EC34F0E55258
:10209000E550226EE550216EE550206EE7501F6E30
:1020A000FC0EE3CFE6FFE3CFE6FFE3CFE6FFE3CFAF
:1020B000E6FF23EBE6FF24EBE6FF25EBE6FF26EB4E
:1020C000E6FFE9EC34F0E552E550266EE550256E6A
:1020D000E550246EE750236E44E91BEBE6FF1CEB52
:1020E000E6FF1DEBE6FF1EEBE6FF1BEBE6FF1CEB3E
:1020F000E6FF1DEBE6FF1EEBE6FF02012D50142765
:102100002E5015232F50162330501723E9EC34F0AE
:1021100029502C272A502D232B502E232C502F238F
:1021200044E90FEBE6FF10EBE6FF11EBE6FF12EBE5
:10213000E6FF0FEBE6FF10EBE6FF11EBE6FF12EB1D
:10214000E6FF2D5018272E5019232F501A233050F8
:102150001B23E9EC34F0295030272A5031232B502F
:1021600032232C50332344E903EBE6FF04EBE6FF74
:1021700005EBE6FF06EBE6FF03EBE6FF04EBE6FF0D
:1021800005EBE6FF06EBE6FF2D501C272E501D2326
:102190002F501E2330501F23E9EC34F029503427F0
:1021A0002A5035232B5036232C50372344E9020183
:1021B00007EB08F208EB09F209EB0AF20AEB0BF263
:1021C000E552E5CFDAFFE7CFD9FF64E9000C000C58
:1021D000ECEC16F031E01AEC16F0D00F056E05505D
:1021E000090802E2070E055E05500F0802E2200E04
:1021F000055E05500F0815E30228E96E000E032066
:10220000EA6EEF50D00F066E0650090802E2070E84
:10221000065E06500F0802E2200E065E06500F080A
:1022200002E2FF0E0AD00538F00B0624E66E38EC09
:1022300016F0E552E750EF6E000E82EF16F0ECEC70
:1022400016F024E03DEC16F0C3DF44E900090BE191
:10225000D950060FDDEC16F0020E45EC16F0B8DF93
:1022600044E9000902E0FF0E12D005500101CF6BD6
:10227000CF6FCE6B0650CE25CC6F000ECF21CD6F29
:1022800038EC16F0CCC1EEFFCDC1EDFF000E82EFB1
:1022900016F027EC16F085E944E81AEC16F048E051
:1022A0003DEC16F0CCDF44E900090BE1D950070FF3
:1022B000DDEC16F0040E45EC16F0C1DF44E9000930
:1022C00002E0FF0E36D0E66A010EE66EE66AE66AC6
:1022D000E66AE66EE66AE66A05EBE6FF06EBE6FF0F
:1022E000E66AE66ADCEC2CF0DCEC2CF0E552E5CF9B
:1022F000CFF1E5CFCEF1E5CFCDF1E7CFCCF107EBD4
:10230000D0F108EBD1F10101D26BD36BD051CC27C6
:10231000D151CD23D251CE23D351CF2338EC16F057
:10232000CCC1EEFFCDC1EEFFCEC1EEFFCFC1EEFFBF
:10233000000E45E9E7CFD9FF120027EC16F085E93A
:102340001AEC16F010E01AEC16F0300804E138EC44
:1023500016F0EF6A08D01AEC16F0310806E138ECF6
:1023600016F0010EEF6E000E01D0FF0E41E9E7CF2F
:10237000D9FF120027EC16F081E942E8670E016EE2
:10238000010E026E7BEC16F00101CF6BCEBFCF6960
:10239000CEC1E6FFCFC1E6FF1FEC3BF04FEC16F0DD
:1023A00004E0012A000E0222EDD77BEC16F0CF6B81
:1023B000CEBFCF69CEC1E6FFCFC1E6FF3DEC3BF01B
:1023C0004FEC16F004E0012A000E0222EED701EBDA
:1023D000F3FF02EBF4FF82EF16F0140E6F6E0201B2
:1023E000A66B0201A76B0201A86B2CEC16F0D4ECD3
:1023F00016F00101876BC86BCB6BC96BCA6B1200FF
:102400001F0E0101D8808755E66E87C1CCF101010E
:10241000CD6BCCBFCD69670ECC27010EE1EC16F079
:1024200076EC31F043E912000001E35106E1DBDB19
:10243000A7EC31F042E90201B46B1200FF00120078
:1024400027EC16F081E963E80168D4EC16F001018D
:102450006751510A01E1F8D1010A01E1E8D1020A0C
:1024600001E188D1010A01E153D1100A01E132D121
:10247000040A01E1D7D0110A0EE01E0A01E02AD3B6
:10248000016A200EE66E730EF6EC16F045E90101C6
:10249000010ECB6F1FD36851520A01E1B3D01F0A5E
:1024A00001E18ED00F0A01E17AD00A0A6DE00E0A2E
:1024B00060E0090A53E01C0A42E0030A31E0040A22
:1024C00026E0100A13E0080A01E004D3C00EE66E0D
:1024D000000E9DDBC00EE66E000EE66E010EC1EC36
:1024E00016F0C0C0E6FF30EC2AF00FD0C10EE66E49
:1024F000000E8DDBC10EE66E000EE66E010EC1EC25
:1025000016F0C1C0E6FF18EC2BF041E9E3D2C20E91
:10251000E66E000E7CDBC20EE66E000EE66E70D03C
:10252000ADEC16F001E1051C04E004EBC3F005EB93
:10253000C4F0010EE66EC30EE66E000E70D0ADEC78
:1025400016F001E1051C04E004EBC5F005EBC6F054
:10255000010EE66EC50EE66E000E61D0E7DB05E00B
:1025600002500001C799E8B0C7890001C7B921D05E
:1025700023D0DCDB05E002500001C79BE8B0C78B2D
:102580000001C7AB19D015D0D1DB05E00250000126
:10259000C79DE8B0C78D0001C7AD0ED00AD0C6DB1D
:1025A00005E002500001C79FE8B0C78F0001C7AF28
:1025B00003D00101310E02D00101300E886F8AD2A2
:1025C0000268D950020F0CDB03DE44E9016EFF0EF6
:1025D000025C0BE002500001070BF36EF80EC7150A
:1025E000F310C76F0101010EC86F0001C751070B3F
:1025F000026E010EE66ED950020FE66EDACFE6FFEC
:10260000010EB6D0AADB01E1051C04E004EB46F2A2
:1026100005EB47F2010EE66E460EE66E020EE66E22
:10262000020EA6D0016A6851580A4FE00A0A3AE041
:10263000040A2DE01F0A27E01D0A21E0170A1BE00B
:102640000E0A0EE00A0A01E07AD060DB030E025C9B
:1026500001E340D2E66A0101D9500C0FC9DAF6D77E
:1026600055DB030E025C01E335D2E66A0101D95065
:10267000180FBEDAF6D7B7DA3FEC2EF00BD0B3DA8C
:1026800002EC2EF007D0AFDA17EC2EF003D0ABDA65
:102690002FEC2EF0F3CFE6FFF4CFE6FFE3EC37F0BC
:1026A00044E918D294DB5DEC34F045E902C2E6FF60
:1026B00003C2E6FF030E9DDB2DEC36F045E906C2B2
:1026C000E6FF07C2E6FF020EA9D0F80EE66E720E14
:1026D0008DDBABD0016A680EE66EE66A600EE66ED0
:1026E000000EE66ED60EE66E750EE66E9EEC1DF0E2
:1026F00046E90101C85104E0F3EC1CF00101C86B8C
:10270000C951CA1101E1E6D1020EC96FCA6BE2D10B
:10271000300E695D026E0250090802E2070E025E89
:1027200002500F0802E2200E025E02500F0801E282
:10273000D1D1016A68514D0A0FE00A0A02E001682E
:10274000C9D124DB900E0101CC27000E69DA900E6E
:102750000101CC27000E0AD019DB600E0101CC2745
:10276000000E5EDA600E0101CC27000E2ADB040E9B
:1027700008DBB0D1D950040F33DA61DD44E9016ED2
:10278000015001E0A7D10001C751070B010A3CE04D
:10279000010A3AE0020A1BE0010A07E0070A01E029
:1027A00099D12DDA0CEC1FF032D029DA0CEC1FF0A5
:1027B00046E9EE0EE66E720E1FDB88DA040E19DBB8
:1027C0008ADA040EE66E8D0EE66E010E2BD009DB62
:1027D00079DA74DA71EC1FF046E9026A060E025CDF
:1027E00010E2090E0202F350036EE66A0101D950AD
:1027F0000C0FA2DA0350B8DA76DA200EEF6E022A56
:10280000EDD771DAEF6A66D1FAD9A9EC1EF046E984
:10281000DEDA5CDA030EEDDA5EDA030EE66E8C0EBB
:10282000E66E010EE66E66EC36F045E953D1520EC7
:10283000685D01E04FD1470E695D01E04BD1010EAB
:10284000C96FCA6B016A46D1D60EF66E750EF76E69
:102850000900F5CF60F00900F5CF61F00900F5CF70
:1028600062F00900F5CF63F00900F5CF64F00900CC
:10287000F5CF65F00900F5CF66F00900F5CF67F0F8
:102880000900F5CF68F00900F5CF69F00900F5CF30
:102890006AF00900F5CF6BF00900F5CF6CF0090084
:1028A000F5CF6DF00900F5CF6EF00900F5CF6FF0B0
:1028B0000900F5CF70F00900F5CF71F00900F5CFF0
:1028C00072F00900F5CF73F00900F5CF74F009003C
:1028D000F5CF75F00900F5CF76F00900F5CF77F068
:1028E0000900F5CF78F00900F5CF79F00900F5CFB0
:1028F0007AF00900F5CF7BF00900F5CF7CF00900F4
:10290000F5CF7DF00900F5CF7EF00900F5CF7FF01F
:102910000900F5CF80F00900F5CF81F00900F5CF6F
:1029200082F00900F5CF83F00900F5CF84F00900AB
:10293000F5CF85F00900F5CF86F00900F5CF87F0D7
:102940000900F5CF88F00900F5CF89F00900F5CF2F
:102950008AF00900F5CF8BF00900F5CF8CF0090063
:10296000F5CF8DF00900F5CF8EF00900F5CF8FF08F
:102970000900F5CF90F00900F5CF91F00900F5CFEF
:1029800092F00900F5CF93F00900F5CF94F009001B
:10299000F5CF95F00900F5CF96F00900F5CF97F047
:1029A0000900F5CF98F00900F5CF99F00900F5CFAF
:1029B0009AF00900F5CF9BF00900F5CF9CF00900D3
:1029C000F5CF9DF00900F5CF9EF00900F5CF9FF0FF
:1029D0000900F5CFA0F00900F5CFA1F00900F5CF6F
:1029E000A2F00900F5CFA3F00900F5CFA4F009008B
:1029F000F5CFA5F00900F5CFA6F00900F5CFA7F0B7
:102A00000900F5CFA8F00900F5CFA9F00900F5CF2E
:102A1000AAF00900F5CFABF00900F5CFACF0090042
:102A2000F5CFADF00900F5CFAEF00900F5CFAFF06E
:102A30000900F5CFB0F00900F5CFB1F00900F5CFEE
:102A4000B2F00900F5CFB3F00900F5CFB4F00900FA
:102A5000F5CFB5F00900F5CFB6F00900F5CFB7F026
:102A60000900F5CFB8F00900F5CFB9F00900F5CFAE
:102A7000BAF00900F5CFBBF00900F5CFBCF00900B2
:102A8000F5CFBDF00900F5CFBEF00900F5CFBFF0DE
:102A90000900F5CFC0F00900F5CFC1F00900F5CF6E
:102AA000C2F00900F5CFC3F00900F5CFC4F009006A
:102AB000F5CFC5F00900F5CFC6F00800F5CFC7F097
:102AC000C86BCB6B010EC91904E1CA5102E1C96B95
:102AD000CA6B016A015064E9E7CFD9FF1200B7D889
:102AE00081E943E88DDC016E015042E00A0EE66E9A
:102AF000670EE66E010EE66E49EC34F043E9F350E2
:102B0000026EF450036E0150010187271F0EE76E1D
:102B1000871902E7E73402D0E750875D09E3010E29
:102B2000F36EF46AF3508708026E010EF454036EDC
:102B3000025003101DE002EBE9FF03EBEAFFEF6A2E
:102B40007FDC000906E0430EE66E7C0EE66E000EAA
:102B500005D03E0EE66E7C0EE66E000E4AD92DECD8
:102B600034F045E90101876B77D80201010EB46F9B
:102B70000201B45101E058DC44E9E7CFD9FF12006B
:102B80000CEC37F02EEC37F00201A651030827E2D7
:102B9000060EA65D24E3A3DFD2EC31F00101CA35B5
:102BA00008E2C9510108000ECA5503E2C92B000E04
:102BB000CA230A0EC91913E1CA5111E1E668E66A8F
:102BC000F2EC1DF042E92CEC37F00101C96BCA6B45
:102BD000C907000ECA5BC951CA11FAE12FDC120005
:102BE000ECD8CDEF16F0880EE66E010EE66E120000
:102BF000A3D8090E0202F350B7D8022A1200F1D866
:102C0000D950060FDAD8D950040FDDEF16F0E66E72
:102C1000C4D8E8EC10F044E9016E010EE66E120033
:102C2000D0D8BBD849EC11F044E9016E010EE66E34
:102C3000C6EF16F002EBE9FF03EBEAFFEF501200DC
:102C40009DEC11F044E9016EFF0E025C1200D9CF39
:102C5000E6FFE1CFD9FF1200200EE66EE66AE66AD3
:102C6000670EE66E010EE66EEFEC33F045E91200FA
:102C700000EBE9FF01EBEAFF1200D950050F9DD8E8
:102C800002EBE6FF03EBE6FF120001010224CC6F2A
:102C9000000E0320CD6FCCC1E6FFE66E120042E9C4
:102CA000F3CFCCF1F4CFCDF10101F350F4101200C9
:102CB0001FEC11F044E9016E041C1200D9500C0FF6
:102CC000DDEF16F0D950180FDDEF16F05DEC34F0A3
:102CD00045E9F1EF16F02DEC36F045E906EBE6FF9D
:102CE00007EBE6FF1200080E0324EA6A880FE96E7C
:102CF000010EEA22120001EBE9FF02EBEAFFEFCF3F
:102D0000CEF1120043E9E7CFD9FF1200030EE66EC1
:102D1000010EE66ED3DFD6DFF8EC1CF046E9050EB7
:102D2000E66E730E63D845E9026A12000268D95054
:102D3000020F56DF20EF16F0CE6FDACFCFF1025040
:102D4000040DCE51F324CC6FDA50F420CD6FCCC1FA
:102D5000E6FFE66E040EE66E120004680568D950C0
:102D6000040F3EDF58EF16F0D16B880FD06F010EC5
:102D7000D123D0C1E6FFD1C1E6FF8BEC36F046E9A6
:102D8000120037D88BEC36F046E912000250040DE1
:102D9000F3CFCCF1F4CFCDF11200BAEC11F0F3CFB8
:102DA000E6FFF4CFE6FF1200400EE66EE66AE66A42
:102DB0001ADFEFEC33F045E91200E66EDACFE6FFFA
:102DC0001200CD23CCC1E6FFCDC1E6FF1200FD0EFF
:102DD000E66E720EFCEF16F03ADF85E942E81AEF74
:102DE00016F004EBE6FF05EBE6FF120005D85DEFF9
:102DF00034F0E66EF3EF15F0E66EE66AF3EF15F0E9
:102E000000000000000000000000000000000000C2
:102E100000000000000000000000000000000000B2
:102E200000000000000000000000000000000000A2
:102E30000000000000000000000000000000000092
:0839B8000201000E886F050EEC
:1039C000896F020EE66EF00EE66E460EE66E020E91
:1039D000E66E52D944E90201461D04E1471D02E1A9
:1039E000466B476B12000201466B476BDFEF1FF01F
:1039F000EBDB41E8076AD890075002E6030E075C4C
:103A000045E200EBE9FF01EBEAFF6FDB0101D56B5B
:103A1000D4BFD569FFDACFAF02D0D069D1690D0E1E
:103A20001F0B03E0010168DBFEE107EBCCF10101B4
:103A3000CD6BCCBFCD6941DB0224E96ECD510320B3
:103A400006DB00EBE9FF01EBEAFF060EE926000EBC
:103A5000EA224BDBD56BD4BFD569DCDACFAF02D01D
:103A6000D069D1690E0E1F0B03E0010145DBFEE1B9
:103A700007EBCCF10101CD6BCCBFCD691EDB04247B
:103A8000E96ECD510520E3DA072AB5D742E9E7CF41
:103A9000D9FF1200D9CFE6FFE1CFD9FF85E942E88F
:103AA00002EBF6FF03EBF7FFF86AA68EA69CA6844E
:103AB000A688F250800B01E0010E066EF29E550EB4
:103AC000A76EAA0EA76EA68200000650E8B0F28E7E
:103AD000E8A0F29EA694056A400E055C2BE2055014
:103AE0000024E96E000E0120EA6EEF50F56E0D0025
:103AF00005281F0B1DE1200EF65E000EF75A000E82
:103B0000F85AA68EA69CA684A698F250800B01E0D7
:103B1000010E066EF29E550EA76EAA0EA76EA68225
:103B20000000A694200EF626000EF722000EF822C2
:103B3000052AD2D743E9E7CFD9FF120045DB7FE85A
:103B400045E83F0E0414076EC00E0414086EFF0E05
:103B50000514096E400EE66EE66A08EBE6FF09EB17
:103B6000E6FFE66AD9500B0F24DBCCEC33F047E9D3
:103B70000050011026E0D890075002E6400E075C86
:103B800020E2C1DAEF50E66E0101D9500B0FCC6F85
:103B9000DACFCDF107EBCEF1CF6BCEBFCF69CC51F1
:103BA000CE25E96ECD51CF21EA6EE552E750EF6E9A
:103BB000072A042A000E0522022A03220006015ABF
:103BC000D7D7D9500B0FF5DA08EBE6FF09EBE6FF84
:103BD00061DF44E900500110B4E17FE946E9E7CF35
:103BE000D9FF1200D9CFE6FFE1CFD9FF83E941E841
:103BF000A6A202D00000FCD700EBA9FF01EBA8FFB2
:103C0000A69EA69CA698A684F250800B01E0010E09
:103C1000036EF29E550EA76EAA0EA76EA6820350E3
:103C2000E8B0F28EE8A0F29EA69442E9E7CFD9FF71
:103C30001200EBD984E900EBA9FFA69EA69CA68002
:103C400001EBE9FF02EBEAFFA8CFEFFF61D2DDD97C
:103C500085E9005010E003EBE6FF01EBE9FF02EB22
:103C6000EAFFEFCFE6FFBEDF42E90006012A000EC1
:103C70000222032AEED74CD2C8D985E943E882EB69
:103C800005F083EB06F081EB07F0A6B2FED7A19812
:103C900000500EE007EBE6FF05EBE6FF06EBE6FF64
:103CA000C8DF43E90006052A000E0622072AF0D7DE
:103CB00044E9E7CFD9FF1200A8D989E942E8020117
:103CC0004651DC08050E475502E2466B476BB50EC0
:103CD000E66EE66A06EBE6FF07EBE6FFA8EC2CF0E3
:103CE000E552E5500A6EE750096E5A0E01010224B2
:103CF000CC6F000E0320CD6FCC510926CD510A2286
:103D0000020EE66ED950090F54DA020EE66EE66A2C
:103D1000A8D95DDAA6D909DA0101CC51CD1114E197
:103D2000400EE66EE66A16D9400ECC5F000ECD5B03
:103D3000010E88D9FEE115DA200ECC5F000ECD5BB6
:103D4000010E80D9FEE137D93AD943E9E7CFD9FF4F
:103D500012003ADA42E8C00E87D9C00EB6D910E197
:103D6000CF51CD190DE102014651005C4751015878
:103D700007E2020EE66EE66EE66A400E2BD90BD025
:103D8000CBD9010ED890F636F736E806FBE109DA12
:103D90000A00F550086EB50E71D9C7D901015A0E47
:103DA000CC5F000ECD5BAFD9CCC1EEFFCDC1EDFF36
:103DB000B50EE66EE66A62D90101FE0EE350075CBD
:103DC000CE6F41E9E5500858CF6FCEC1E6FFE66EF1
:103DD000E7EC2BF0AAD904EBE9FF05EBEAFFCCC135
:103DE000EEFFCDC1EDFF43E9E7CFD9FF12000DD9BA
:103DF00074D902E2466B476B49D9FAD847D9BDD886
:103E000009E1C8D91FD9FEE1ACD9100E51D91AD990
:103E1000FEE1D1D8D4D885D1D7D944E8E00E24D951
:103E2000E00E53D910E1CF51CD190DE102014651F9
:103E3000005C4751015807E2040EE66EE66EE66A42
:103E4000200EC8D80BD068D9020ED890F636F736B7
:103E5000E806FBE1EFD80800F5500A6E54D909EBEB
:103E6000EEFF0AEBEDFF04EBE9FF05EBEAFF07EBE2
:103E7000EEFF08EBEDFF55D1C8D82FD902E2466B13
:103E8000476B0DD9B5D80BD978D809E183D9DAD8E1
:103E9000FEE167D9100E0CD9D5D8FEE18CD88FD8A9
:103EA00040D1B3D883E90C0E88D946C2CCF147C2C1
:103EB000CDF10101CD03F3CFCDF1CC03F3CFCCF1A4
:103EC000F450CD27000E53D90201462B000E472394
:103ED000FA0E465D000E475902E3466B476B6FD8FA
:103EE00017D172D94CE818D90C0EF702F3CFF7FFAF
:103EF000F602F3CFF6FFF450F7269CD80900F550F0
:103F00000A6E0900F5500B6E0900F5500C6E0900A1
:103F1000F5500D6E0900F5500E6E0900F5500F6E4C
:103F20000900F550106E0900F550116E0900F550AA
:103F3000126ED950070F3DD904EBE6FF05EBE6FF03
:103F400002EBE6FF03EBE6FF53DD46E94DE9E7CF81
:103F5000D9FF1200480EE66E020EE66E8DDE44E9D1
:103F6000400EE66EE66A480EE66E020EE66E46C249
:103F7000CCF147C2CDF10101120000EBE6FF01EBED
:103F8000E6FF02EBE6FF03EBE6FFDDD80B6ECF5159
:103F90000C6E040EE66ED950090F0BD9040EE66EB6
:103FA000E66A200EC8D813D9200EC5D8BED80101A4
:103FB000CC51CD111200000E0101B7EF20F0020E1E
:103FC000E66E460EE66E020EE66EF00EE66E3FDE22
:103FD00044E91200F2D8EAEC2BF0A8EC2CF0A5D8BA
:103FE000CCC1E6FFD950070FE4D846DE44E9120001
:103FF00004EBE6FF05EBE6FF06EBE6FF07EBE6FF6B
:10400000A2D8096ECF510A6E1200D9CFE6FFE1CFD8
:10401000D9FF1200D890D437D537D251D425E96EC4
:10402000D351D521EA6EEECFCEF1EFCFCFF1D06BE9
:10403000D16B1200B6D80900F550086E0900F55092
:10404000096E1200D890CC37CD37E8061200EA6E20
:10405000CEC1EEFFCFC1EEFFD0C1EEFFD1C1EEFF6A
:104060001200400E9BEF20F0020146150101CC6FBB
:10407000FF0E020147150101CD6F1200E66EE66AE0
:1040800007EBE6FF08EBE6FFEAEF2BF0E0C1E6FF07
:10409000E1C1E6FFE2C1E6FFE3C1E6FF1200DCC1D9
:1040A000E6FFDDC1E6FFDEC1E6FFDFC1E6FF12008D
:1040B000CC5F000ECD5B020E1200D890CC37CD370E
:1040C000D890CC37CD37CC5112000014CE6FFF0EF4
:1040D0000114CF6FCE51CC19120089E944E80201D6
:1040E0004651EE08020E47551200E9CFD2F1EACF51
:1040F000D3F107EBD4F11200D890CE37CF37D037B9
:10410000D137E806120002EBE9FF03EBEAFF1200E9
:1041100041E9E7CFD9FF120000EBF6FF01EBF7FF13
:10412000120045E9E7CFD9FF1200E552E5CFCDF106
:10413000E7CFCCF11200E66EE66A46C2E6FF47C260
:10414000E6FFEAEF2BF0DDEC34F048E9A2C2CCF157
:10415000A3C2CDF1A4C2CEF1A5C2CFF10101CE51CF
:10416000120029DF400EE66EE66EAAEF1FF0CC27A4
:104170002E0ECD23CCC1E6FFCDC1E6FFDFDC46E944
:104180001200CCC1E6FF63DD44E90201462B000EBC
:1041900047231200400EE66EE66ADCDE200E58EF82
:1041A00020F0000EF6262E0EF7220900F550076EBD
:1041B0001200E66EDACFE6FF1200E66EE66A00EB6A
:1041C000E6FF01EBE6FF120020DF87E91200A8EC12
:0841D0002CF0ABDFC1EF20F081
:0841D800800EC76E280EC66EB2
:1041E000180EC86EC56A800EE66E080EE66E0CEC00
:1041F0003DF042E90101636B646B006B016B010EE2
:10420000026F656B666B8A8A8996536B546B556B2C
:10421000566B53C14FF154C150F155C151F156C1C4
:1042200052F153C14BF154C14CF155C14DF156C13E
:104230004EF1120074DA82E941E80050E824900F50
:10424000026EC0EC15F011EC3EF0C580C5B0FED793
:1042500002EBE6FF72DAC5AC02D0000E07D09F0E6B
:10426000E66E6BDAC584C5B4FED7010EF36EF46A50
:1042700042E9E7CFD9FF120052DA84E946E802505A
:10428000E824910F046E800E076EC0EC15F011EC5F
:104290003EF0C580C5B0FED704EBE6FF4EDAC5BCE4
:1042A00027D0030EE66ED950050FE66EDACFE6FF93
:1042B000DFEC3BF043E911EC3EF0C58AC588C5B898
:1042C000FED7C584C5B4FED705EBCEF1CEC1CFF184
:1042D0000101CE6B0650CE25CC6F000ECF21CD6FE5
:1042E00000EBE9FF01EBEAFF2DDA800E071402E094
:1042F000000E01D0010E47E9E7CFD9FF12000FDA17
:1043000082E90C0EE66E7F0E0014FE0BFD0BE66ECE
:10431000AD0EE66EB0EC3BF043E9010E18DA3AEC74
:104320003EF041E9E7CFD9FF1200F9D981E942E82F
:10433000EAEC3DF0000EF35C016E020EF458026EE2
:1043400031EC3EF001EBF3FF02EBF4FF43E9E7CF82
:10435000D9FF1200050E00DA020EFED9010EFCD9BB
:10436000970EE66ECCDF41E91200D9D981E941E828
:1043700026DA01E13CD12ADA01E139D12EDA01E174
:1043800036D10101005113E05DC157F15EC158F112
:104390005FC159F160C15AF161C15BF162C15CF169
:1043A0008A9A030ED4D989860101006B1CD1016A57
:1043B000D890015002E6030E015C01E3FAD088D9DF
:1043C000E9BEEA6889D9570EE926010EEA22EECF46
:1043D000D2F1EFCFD3F17CD9E9BEEA687DD95D0E89
:1043E000E926010EEA22EE500101D25DD06FEE50B7
:1043F000D359D16FD06DD11F000ED12384D9060EB1
:10440000E926000EEA2290D9CEBFCF696ED9E668C0
:10441000E668E668E66863C1D4F164C1D5F1D66B9D
:10442000D76BD5AF02D0D669D769D4C1E6FFD5C165
:10443000E6FFD6C1E6FFD7C1E6FF4AD9E9BEEA6882
:104440004BD94AD93F0EE926010EEA2289D988D9EB
:1044500023EC2CF0DCEC2CF0E552E5CFD3F1E5CFEA
:10446000D2F1E5CFD1F1E7CFD0F14DD95DD9CEBFB3
:10447000CF693BD92DD9E9BEEA682ED92DD94B0E8B
:10448000E926010EEA22EE6AEE6AEE6AEE6A20D9A9
:10449000E9BEEA6821D9150EE926010EA5D9E9BEC3
:1044A000EA681AD9210EE926010EEA2280D9E9BE6E
:1044B000EA6812D92D0EE926010E70D9E9BEEA6824
:1044C0000BD9390EE926010E5DD9E9BEEA68FD0E69
:1044D000E926000EEA22EFCFCEF1CF6BCEBFCF6937
:1044E00044D9E9BEEA6887D92DD9F2D8E9BEEA688D
:1044F000F3D80F0EE926010E77D9E9BEEA68ECD8A9
:104500001B0EE926010EEA22010151D9E9BEEA6833
:10451000E3D8270EE926010E41D9E9BEEA68DCD8C6
:10452000330EE926010E2ED9E9BEEA68FA0EE92615
:10453000000EEA22EFCFCEF1CF6BCEBFCF6915D9F7
:10454000E9BEEA68C9D8030EE926010EEA22FAD8C4
:104550000001C751800B24E0BBD8E9BEEA684BD903
:10456000FFD813EC36F042E9F3CFCCF1F4CFCDF124
:10457000140E0101D890CDBF03D0CC5D000ECD59F3
:104580000FE2010E01EBF3FF015204E0D890E83690
:10459000F306FCE101016511656F030E662707D084
:1045A0000101665102E0660501D0000E666F012A26
:1045B000FFD6665101E1656B8996030EC8D88A8AD9
:1045C0000101010E006F030EE66E010EE66E48EC6F
:1045D00024F042E90101636B646B022B0251040871
:1045E00002E2010E026FB6DE0101016B19D001017A
:1045F000643516E263516408000E645511E2100E32
:10460000656FDDD802E101016581E0D802E10101B9
:104610006583E3D802E10101658501010A0E666F39
:1046200029EC3EF0000950E180DEF3CFCCF1F4CF6D
:10463000CDF10101CE6BCF6BCDAF02D0CE69CF698A
:1046400001010151040DF3CFE9FFF4CFEAFF4B0E56
:10465000E926010EEA220101CC51EE26CD51EE22CF
:10466000CE51EE22CF51EE220101012B030E015D4E
:104670001CE3016B4BC13FF14CC140F14DC141F115
:104680004EC142F14FC143F150C144F151C145F116
:1046900052C146F153C147F154C148F155C149F1E6
:1046A00056C14AF1632B000E64230151020A08E04F
:1046B000030A04E0010A08E1970E03D08F0E01D02F
:1046C000870EE66E1CDE41E942E9E7CFD9FF120012
:1046D00001EBE9FFEA6A1200D890E936EA361200E7
:1046E000E66ECADD43E900091200D890CE37CF3715
:1046F000CC51CE25E96ECD51CF21EA6ED0C1EEFF6F
:10470000D1C1EDFF1200010102510C0DF3CFE9FF01
:10471000F4CFEAFF030EE926010EEA221200D9CFF8
:10472000E6FFE1CFD9FF1200E9CFCCF1EACFCDF11E
:1047300001EBCEF10101CF6B120033EC3CF041E90B
:1047400011EF3EF0CCC1EEFFCDC1EDFF1200E66EE1
:10475000F6EC3DF041E91200E66E6CDD41E9120035
:10476000EECFE6FFEECFE6FF1200CEC1E6FFCFC1EF
:10477000E6FFA8EC2CF0E552E5CFCDF1E7CFCCF188
:1047800068EF23F0EA22D251EE24D06FD351EE200D
:10479000D16FD0C1E6FFE66E68EF23F0EA22D45174
:1047A000EE24D26FD551EE20D36F68EF23F0D651AF
:1047B000EE24D46FD751EE20D56F68EF23F05D0E55
:1047C000E66E010EE66E050E70EF23F05F0EE66EEC
:1047D000010EE66E020E70EF23F0610EE66E010E22
:1047E000E66E010E70EF23F0EA22EECFD6F1EFCFA6
:1047F000D7F168EF23F070DF090EE926010EEA22F7
:024800001200A4
:0E480200D6DA83E941E8036AD890035002E653
:10481000180E035C39E2040EE66E03EBE6FF84EC4F
:104820002CF041E9E750000906E00101D06BD16BA3
:10483000D26BD36B06D00101D06BD16BD26B010E62
:10484000D36F00EBE9FF01EBEAFFE9CFCCF1EACF50
:10485000CDF103EBCEF1CF6BCEBFCF69D890CE3781
:10486000CF37D890CE37CF37CC51CE25E96ECD514A
:10487000CF21EA6ED0C1EEFFD1C1EEFFD2C1EEFF73
:10488000D3C1EEFF032AC1D742E9E7CFD9FF120017
:104890008FDA83E945E8036AD890035002E6060EF2
:1048A000035C0EE203EBE9FFEA6AE9BEEA68A8DA14
:1048B00003EBE9FFEA6AE9BEEA68A5DA032AECD766
:1048C000E66A00EBE6FF01EBE6FF1BEC0CF043E9C8
:1048D0002CC2CCF12DC2CDF12EC2CEF12FC2CFF120
:1048E000020130510101CC27020131510101CD23D8
:1048F000020132510101CE23020133510101CF23C4
:104900003CDA06DA89EC35F044E949DA0ADA00DA09
:1049100058DAE5D9010131DA39DA14C2E6FF15C2F5
:10492000E6FF16C2E6FF17C2E6FF18C2E6FF19C28D
:10493000E6FF1AC2E6FF1BC2E6FF54DAA2C200F28B
:10494000A3C201F2A4C202F2A5C203F2020103351E
:1049500004E3680E0227010E032318DAD9D91CC21A
:10496000E6FF1DC2E6FF1EC2E6FF1FC2E6FF3ADAFF
:10497000A2C204F2A3C205F2A4C206F2A5C207F2C3
:1049800046E9E7CFD9FF120013DA81E94CE8056A5E
:10499000066A076A086A0A6A0B6A060ED8900BBE96
:1049A00003D00A5C000E0B580EE20AEBE9FF0BEB9A
:1049B000EAFF26DA0AEBE9FF0BEBEAFF24DA0A2A20
:1049C000000E0B22EAD70A6A0B6A380ED8900BBE8B
:1049D00003D00A5C000E0B5801E38CD00AEBE6FF13
:1049E0000AEBCEF10BEBCFF101010C0ECF03F3CFAD
:1049F000CFF1CE03F3CFCEF1F450CF27020188518F
:104A00000101F324CC6F020189510101CF21CD6F47
:104A1000CCC1E6FFE66E1BEC0CF043E9100ED8901B
:104A20000BBE03D00A5C000E0B5860E2030E0101BE
:104A30000A14CC6FCD6B030ECC1958E1CD5156E161
:104A4000096AD890095002E6030E095C4FE2020E93
:104A5000E66EE66AE66AE66AB0D9E9BEEA6833D984
:104A6000C8D9EFCFE6FF23EC2CF0E552E5CFEDFF00
:104A7000E5CFEDFFE5CFEDFFE7CFEFFF9ED9E9BE34
:104A8000EA6821D9EE50016EEE50026EEE50036ED0
:104A9000EF50046E92D9E9BEEA68BDD98ED9E9BE5D
:104AA000EA6893D901EBD0F102EBD1F103EBD2F13B
:104AB00004EBD3F182D9E9BEEA680BD944D9D950C5
:104AC000050FE96EDACFEAFFCC51EE26CD51EE228A
:104AD000CE51EE22CF51EE2270D9E9BEEA6893D9C9
:104AE0006CD9E9BEEA688CD9092AABD70A2A000E2C
:104AF0000B226BD7030E0C6ED8900C5002E6060EFC
:104B00000C5C47E2EDC1E6FFEEC1E6FFEFC1E6FF58
:104B1000F0C1E6FF0CEBE9FFEA6AE9BEEA6855D9A5
:104B20000CEBE9FFEA6AE9BEEA6875D901EBE6FF3A
:104B300002EBE6FF03EBE6FF04EBE6FF42D92FD9D9
:104B40000CEBE9FFEA6AE9BEEA68C3D80101FBD8C9
:104B5000F1D8D950010FE96EDACFEAFF020EE76E05
:104B6000D890030EEB32020EEB32010EEB32EF3235
:104B7000E706F6E1D950050FE96EDACFEAFF0150FA
:104B8000EE260250EE220350EE220450EE220C2AB2
:104B9000B3D705EBA2F206EBA3F207EBA4F208EB06
:104BA000A5F24DE9E7CFD9FF120030D92ADE42E95C
:104BB0009FD8EADEA2C20CF2A3C20DF2A4C20EF28A
:104BC000A5C20FF20201106B116B200E126F136B56
:104BD0001200EED882E945E80201105111111211BC
:104BE000131165E0005002E1010E456F066AD8908E
:104BF000065002E6180E065C4AE27AD800500EE033
:104C000006EBE9FFEA6AE9BEEA68AAD8EE26115186
:104C1000EE221251EE221351EE220DD006EBE9FFE7
:104C2000EA6AE9BEEA689CD8EE5E1151EE5A12516A
:104C3000EE5A1351EE5AA8DE52D80101CC51026E41
:104C4000CD51036ECE51046ECF51056E02010C5151
:104C5000025C0D5103580E5104580F51055815E2CE
:104C6000600EE66EE66A600EE66E000EE66ECED868
:104C7000A1EC33F046E902EB0CF203EB0DF204EB8E
:104C80000EF205EB0FF20201456B062AB0D7455133
:104C90000DE000500BE0010E1F0B08E00201D89060
:104CA0001333123311331033E806F9E121D80CC263
:104CB000A2F20DC2A3F20EC2A4F20FC2A5F246E9FF
:104CC000E7CFD9FF120087D8140EE926020EEA2298
:104CD000120081D82C0EE926020EEA221200A2C28E
:104CE000CCF1A3C2CDF1A4C2CEF1A5C2CFF1120086
:104CF000600EE66EE66A8AD8600EE66E000EE66E1C
:104D0000A1EC33F046E9120074D8EECFE6FF1200B2
:104D100004EBE6FF05EBE6FF06EBE6FF07EBE6FF3D
:104D20001200A2C2E6FFA3C2E6FFA4C2E6FFA5C22C
:104D3000E6FF1200CC51016ECD51026ECE51036ED2
:104D4000CF51046E1200D051EE5CCC6FD151EE58B1
:104D5000CD6FD251EE58CE6FD351EE58CF6F1200B7
:104D60003AD8600EE926000EEA2202011051120024
:104D7000EE6AEE6AEE6AEE6A1200CC51046ECD5114
:104D8000056ECE51066ECF51076E1200E9C1E6FFE7
:104D9000EAC1E6FFEBC1E6FFECC1E6FF1200A2C2EA
:104DA000D0F1A3C2D1F1A4C2D2F1A5C2D3F11200B5
:104DB000D9CFE6FFE1CFD9FF120009EBE9FFEA6A9C
:104DC0001200DDEC34F048E9120025D8FADF87DF65
:104DD00001019AEF26F0D890E936EA36D890E93604
:104DE000EA36120083EC27F048E979DF9ADFE1EF39
:104DF00026F0EECFE6FFEECFE6FFEECFE6FF1200A5
:104E000062DFB8EF26F065DFB8EF26F0A00EE66EA1
:0C4E1000070EE66E120057DF84EF26F05C
:044E1C0005DA89E941
:104E200045E807340CE3C8D993D97BD9046ECD513A
:104E3000056ECE51066ECF51076E010E0D6E033416
:104E40000CE327DA006ECD51016ECE51026ECF51C8
:104E5000036E010ED8800D540D6E02EBD0F103EB02
:104E6000D1F10101D26BD36BD1AF02D0D269D3693A
:104E7000D0C1E6FFD1C1E6FFD2C1E6FFD3C1E6FF54
:104E800067D923EC2CF0E9D9080E1F0B08E00101CB
:104E9000D890CC37CD37CE37CF37E806F9E10101CE
:104EA000CC5171D90D5001E0E2D909EBA2F20AEB25
:104EB000A3F20BEBA4F20CEBA5F246E9E7CFD9FF86
:104EC0001200B2D985E944E8033409E200EBA2F20A
:104ED00001EBA3F202EBA4F203EBA5F210D0D9D9B7
:104EE000056ECD51066ECE51076ECF51086E05EBA3
:104EF000A2F206EBA3F207EBA4F208EBA5F245E958
:104F0000E7CFD9FF120090D989E959E8216A20D961
:104F1000D8DF44E9B1D9A2C2E6FFA3C2E6FFA4C22A
:104F2000E6FFA5C2E6FF1DD9CCDF44E9E552E7CF95
:104F3000CFF1E552E7CFCEF1E552E7CFCDF1E55223
:104F4000E7CFCCF1A2C2D0F1A3C2D1F1A4C2D2F179
:104F5000A5C2D3F10101D335CF51D31908E6D05101
:104F6000CC5DD151CD59D251CE59D351CF5904E353
:104F7000EFD8F7D892D905D0F4D8EAD88ED9010E57
:104F8000216E0C3401E373D9D2D8D1D890D90D6EEB
:104F9000CD510E6ECE510F6ECF51106E1CD9950EA5
:104FA000CC27DB0ECD23020ECE23F90ECF23CC511E
:104FB000FBD8690E156E1F0E166EF30E176E18686D
:104FC00013D948D9BDD807D9050ECC27000ECD235B
:104FD000CE23CF23CC51E8D807D957D9F30E156E7D
:104FE0008E0E166ED30E5DD908D9CA0ECC272E0EA2
:104FF000CD23D80ECE23020ECF230DEBD0F10EEB36
:10500000D1F10FEBD2F110EBD3F1DBD805D9B2D847
:105010003CD99B0E156EA80E166E250E42D9540E65
:10502000156EFB0E166EA40E176E186A0DEBE6FFDA
:105030000EEBE6FF0FEBE6FF10EBE6FF0BD9ECD82B
:10504000DCD8CF2B15EBD0F116EBD1F117EBD2F169
:1050500018EBD3F1B6D8196ECD511A6ECE511B6E26
:10506000CF511C6E19EBE6FF1AEBE6FF1BEBE6FFD8
:105070001CEBE6FF90D8D2DE4FD862D8215012E167
:10508000203408E2B50ED06F1F0ED16F920ED26F92
:10509000010E07D04B0ED06FE00ED16F6D0ED26FA8
:1050A000FE0EC7D807340DE204500008000E055468
:1050B000000E0654000E075404E27ED86CD831D896
:1050C0003FD8033408E3960ED06FC00ED16FDB0ECD
:1050D000D26FFC0EAED8D880205008E7960E1D5C2B
:1050E000C00E1E58DB0E1F58FC0E205809E28ED849
:1050F000D40EEE267E0EEE22480EEE22060EEE2294
:105100001DEBA2F21EEBA3F21FEBA4F220EBA5F223
:105110005AE9E7CFD9FF120048E9AED80101CC51D6
:105120001200DCEC2CF099D80101CC51120009EBF3
:10513000E6FF0AEBE6FF0BEBE6FF0CEBE6FF1200E7
:105140001D6ECD511E6ECE511F6ECF51206E1200BE
:1051500004EBE6FF05EBE6FF06EBE6FF07EBE6FFF9
:10516000120000EBE6FF01EBE6FF02EBE6FF03EBCC
:10517000E6FF120015EBE6FF16EBE6FF17EBE6FF86
:1051800018EBE6FF1200096ECD510A6ECE510B6E80
:10519000CF510C6E12001DEBE6FF1EEBE6FF1FEB7E
:1051A000E6FF20EBE6FF1200116ECD51126ECE51DC
:1051B000136ECF51146E1200E668E668E668E66882
:1051C0001200D051CC27D151CD23D251CE23D3516F
:1051D000CF23CC51120009EBCCF10AEBCDF10BEB54
:1051E000CEF10CEBCFF1120011EBE6FF12EBE6FF74
:1051F00013EBE6FF14EBE6FF120011EBCCF112EB20
:10520000CDF113EBCEF114EBCFF11200D9501D0FFD
:10521000E96EDACFEAFF1200156ECD51166ECE514F
:10522000176ECF51186E1200D9CFE6FFE1CFD9FF2C
:105230001200D36FEBDFEE50D05DCC6FEE50D15942
:10524000CD6FEE50D259CE6FEE50D359CF6FCC51B7
:10525000A0EF28F08FDF57EF29F0E552E5CFCFF12F
:10526000E5CFCEF1E5CFCDF1E7CFCCF11200A4DF51
:105270005EDF57DFC3EF28F0A2C2CCF1A3C2CDF1AD
:10528000A4C2CEF1A5C2CFF1120085DF10D8A0EFE5
:1052900028F092DF66DF91EF28F0C0DD3DDFC3EF3D
:1052A00028F0176E186A43DFD5DFD4EF28F0DDEC65
:0652B00034F08CEF28F041
:0A52B600060EE66EF2EC3CF041E952
:1052C000400EE66E81EC3BF041E9D70E9314936EED
:1052D0000AEC3EF0BA6A8A861200EDD987E98F0E91
:1052E000E66E730EE66EE66A15DA5DEC34F045E9BB
:1052F000D9CFE9FFDACFEAFF080EE76ED890030EA8
:10530000EB32020EEB32010EEB32EF32E706F6E142
:10531000DED9DDD9BED9DDEC34F048E9A2C2D0F146
:10532000A3C2D1F1A4C2D2F1A5C2D3F1A2C2E6FFB9
:10533000A3C2E6FFA4C2E6FFA5C2E6FFDDEC34F09F
:1053400048E9A2C2CCF1A3C2CDF1A4C2CEF1A5C25C
:10535000CFF1A4C2E6FFA5C2E6FF050EE66EDAD9DC
:1053600066EC36F045E9080E7FD9EF6A070E7CD966
:105370002C0EEF6E050E78D9EF50E66E060EC3D9EF
:10538000EF50E66E050EBFD92E0EEF6E41E9E7CF66
:10539000D9FF120090D98BE956E80B6A91D90D0F0D
:1053A000A7D977D9D950170FA3D9850EE66E730EFA
:1053B000A3D95DEC34F045E9D9500D0F73D9D9501C
:1053C000170F70D97F0EE66E730E96D92DEC34F060
:1053D00045E9010E0C6E0CEBCCF10101CD6BCCBF9D
:1053E000CD697ED92A080AE00CEBCCF1CD6BCCBF9D
:1053F000CD6976D90B180B6E0C2AEDD7E66AD95019
:105400000B0F8DD9010EE66E0CEBCEF1CF6BCEBF3C
:10541000CF690850CE25CC6F0950CF21CD6FCC2B52
:10542000000ECD23CCC1E6FFCDC1E6FF8BEC36F0FC
:1054300046E957E9E7CFD9FF12003DD989E972E87B
:1054400028D93ED9090F6BD9A5DF4AE9D950090FF0
:1054500066D959EC3CF042E973E9E7CFD9FF120075
:105460002AD982E9005003E00C0EBA6E02D0BA6A63
:105470008A860028E86CE66EE66A0DEC3CF042E9AC
:1054800041E9E7CFD9FF120016D983E946E8FA0EC1
:10549000036E700E046E050EE66EE66A200E015C69
:1054A0000101CC6FCD6B800B01E0CD69CCC1E6FF73
:1054B000CDC1E6FFA8EC2CF0E552E550076EE750B1
:1054C000066E056A050E055C2EE2005022E0040E11
:1054D000D8800554CFD8086E700E0814E8380F0B2A
:1054E000CD6F070E0814100D080E0814F310CD111F
:1054F000086E440E0814E840E8403F0BCD6F110ED3
:105500000814040DF3CFCCF12A0E0814F310CD11BA
:1055100002D00550AFD8086E08EBE6FF52EC3BF026
:1055200041E9052ACFD747E9E7CFD9FF1200D9CF04
:10553000E6FFE1CFD9FF83E942E8C0EC15F00201B4
:10554000D8800B5104E7C00E0A5DFF0E0B5901E233
:10555000046A02010B3504E20A514008000E0B55A3
:1055600002E2010E046E0001C7AB04D0010ED88028
:105570000454046E0001CA5102E18B9C55D0040E04
:10558000E66EE66A00EBE6FF01EBE6FFF50EE66E7F
:10559000010EE66E84EC34F046E9000945E0050EA4
:1055A000E66EE66A00EBE6FF01EBE6FFF50EE66E5F
:1055B000010EE66EAFEC34F046E98B9C00008B8C5C
:1055C0000000CAC0E6FF34D841E900008B92000019
:1055D0008B80000038EC3EF00000036A040E035C90
:1055E0001EE204500FE0010EE66E030ED880035455
:1055F0000024E96E000E0120EA6EEFCFE6FF44DFE3
:1056000042E90BD0E66A03500024E96E000E012047
:10561000EA6EEFCFE6FF38DF42E9032ADFD700006A
:1056200034EC3EF000008B9043E9E7CFD9FF120045
:10563000D9CFE6FFE1CFD9FF82E98B8200008B80D2
:10564000000038EC3EF00000400E00107F0BE66ECC
:1056500052EC3BF041E9000034EC3EF000008B904E
:1056600041E9E7CFD9FF12000424E96E000E0520BE
:10567000EA6E120001010624CC6F000E0720CD6FE8
:10568000CC510324F66ECD510420F76E0800F5507E
:10569000120000EBE6FF01EBE6FF02EBE6FF03EB97
:1056A000E6FF12003CD808EBE6FF09EBE6FF09EC49
:1056B00034F044E91200D9CFE6FFE1CFD9FF120060
:1056C00029D806EBE6FF07EBE6FFD9501200E0C150
:1056D000E6FFE1C1E6FFE2C1E6FFE3C1E6FF12003B
:1056E000CC510824E96ECD510920EA6EEF5012002A
:1056F00016D8F3DD46E91200E66EE66A08EBE6FF2F
:1057000009EBE6FF1200B0DFE552E750EF6E040E42
:1057100034EF2BF004EBE6FF05EBE6FF1200E66E3C
:06572000DACFE6FF1200E3
:0A57260043E8D9CFE6FFDACFE6FF33
:10573000E1CFD9FFE2CFDAFF89E9066A1200F3DF91
:10574000068001D0F0DF01AEACEF2BF0006C011E43
:10575000E86A012206B0067E03AEB4EF2BF0026CBD
:10576000031EE86A0322067EECEC2BF003BED6EFA4
:105770002BF006AE08D0026C031EE86A0322046C0C
:10578000051EE86A052206B006D084EB00F085EB22
:1057900001F006A004D082EB00F083EB01F0E552AB
:1057A000E5CFDAFFE7CFD9FF45E9000C06BEBBEF36
:1057B0002BF0E9DFFF0C43E8D9CFE6FFDACFE6FFB5
:1057C000E1CFD9FFE2CFDAFF89E9066A1200F3DF01
:1057D000068003D0F0DF01D00682056A046A100E4D
:1057E000E76ED89002360336043605360050045C66
:1057F0000150055805E30050045E0150055A022A85
:10580000E72EF0D706B2120006B006D084EB00F007
:1058100085EB01F006A004D082EB00F083EB01F0F1
:10582000E552E5CFDAFFE7CFD9FF45E9120045E8B9
:10583000D9CFE6FFDACFE6FFE1CFD9FFE2CFDAFF3B
:105840008FE90C6A1200F3DF0C8001D0F0DFE86A08
:1058500003AE34EF2CF0006C011E021E031E012269
:10586000022203220CB00C7E07AE3FEF2CF0046C3A
:10587000051E061E071E0522062207220C7E6CEC62
:105880002DF007BE70EF2CF00CAE0FD0046C051E8F
:10589000061E071EE86A052206220722086C091E5A
:1058A0000A1E0B1E09220A220B220CB00AD088EB1A
:1058B00000F089EB01F08AEB02F08BEB03F00CA017
:1058C00008D084EB00F085EB01F086EB02F087EB6B
:1058D00003F0E552E5CFDAFFE7CFD9FF49E9000C45
:1058E0000CBE46EF2CF0E1DFFF0C42E8D9CFE6FF1B
:1058F000DACFE6FFE1CFD9FFE2CFDAFF86E9036A2C
:105900001200F3DF038001D0F0DF00AE03D0006CA3
:1059100003B0037E01AE02D0016C037E3EEC2DF09D
:1059200001BEA4EF2CF003AE02D0016C026C03B0F8
:1059300081EB00F003A082EB00F0E552E5CFDAFF47
:10594000E7CFD9FF43E9000C03BEEFD7F0DFFF0C30
:1059500044E8D9CFE6FFDACFE6FFE1CFD9FFE2CFC7
:10596000DAFF8AE980EB04F081EB05F082EB06F0C8
:1059700002500402F450016EF350006E0350076EA3
:105980000502F450036EF350026E07500402F35008
:105990000126F4500222E86A032206500502F35061
:1059A0000126F4500222E86A0322E552E5CFDAFF2D
:1059B000E7CFD9FF46E9000C44E8D9CFE6FFDACFBC
:1059C000E6FFE1CFD9FFE2CFDAFF8EE980EB08F006
:1059D00081EB09F082EB0AF083EB0BF00450080234
:1059E000F350006EF450016E04500902F35001268A
:1059F000000EF420026E04500A02F3500226000E3C
:105A0000F420036E04500B02F350032605500802E5
:105A1000F3500126F4500222000E03220550090221
:105A2000F3500226F450032205500A02F3500326D5
:105A300006500802F3500226F450032206500902D1
:105A4000F350032607500802F3500326E552E5CF32
:105A5000DAFFE7CFD9FF48E9000C42E8D9CFE6FFEB
:105A6000DACFE6FFE1CFD9FFE2CFDAFF86E9036ABA
:105A70001200F3DF038003D0F0DF01D00382026A5B
:105A8000080EE76ED890013602360050025C02E341
:105A9000026E012AE72EF7D703B2120003B081EBA2
:105AA00000F003A082EB00F0E552E5CFDAFFE7CF8C
:105AB000D9FF43E9120045E8D9CFE6FFDACFE6FF88
:105AC000E1CFD9FFE2CFDAFF8FE90C6A1200F3DFF2
:105AD0000C8003D0F0DF01D00C820B6A0A6A096ADD
:105AE000086A200EE76ED89004360536063607366B
:105AF000083609360A360B360050085C0150095842
:105B000002500A5803500B5809E30050085E015038
:105B1000095A02500A5A03500B5A042AE72EE4D7B6
:105B20000CB212000CB00AD088EB00F089EB01F047
:105B30008AEB02F08BEB03F00CA008D084EB00F0B2
:105B400085EB01F086EB02F087EB03F0E552E5CF41
:0A5B5000DAFFE7CFD9FF49E91200A0
:065B5A00020EE66EF20EE1
:105B6000E66E9D0EE66E020EE66E3CEC1EF044E91B
:105B70009DC29FF29EC2A0F21200200EE66E310E70
:105B800067D9440EE66EFE0E63D9020EE66ECDECCA
:105B90003DF041E9B40EE66EFE0E5AD987D90201F6
:105BA0009D6BF60E9E6F34EF2FF059D982E944E8D1
:105BB000046A056A020EE66ED950020FE66EDACF6D
:105BC000E6FF00EBE6FF680EE66E1AEC3AF045E9F8
:105BD000000913E1FF0E01010214CD6BCD6FCC6BF8
:105BE000000E0214FF0E0314CF6FCE6FCF6BCE5199
:105BF000CC11046ECD51CF11056E04EBF3FF05EB14
:105C0000F4FF5AD1E66A010EE66E180E70D9F3CF92
:105C1000E6FFF4CFE6FF9FEC2BF0E552E5CFCDF1A8
:105C2000E7CFCCF1CCC1F3FFCDC1F4FF120017D9FF
:105C300081E948E845D9056AC00E066E076A086A18
:105C40000E0E28D905EBE6FF06EBE6FF07EBE6FFB5
:105C500008EBE6FFEAD849E9E7CFD9FF1200FFD801
:105C600081E944E82DD90C0E15D9AAC2E6FFABC2D2
:105C7000E6FFACC2E6FFADC2E6FFD7D81DD1100EDD
:105C800077EF2FF0ECD883E9010101EBCCF1CD6B7C
:105C9000CCC1E6FF100EDCD800EBE6FF110ED8D821
:105CA00041E9E7CFD9FF1200800EE66E080ED0D88A
:105CB000E7D801E0000C010CD2D881E944E8DFDF2D
:105CC000EFD8CE6BCF6BCDAF02D0CE69CF69FDD808
:105CD0009DC2CCF19EC2CDF1CE6BCF6BCDAF02D0C9
:105CE000CE69CF69CF350450CF1908E6CC51015C9D
:105CF000CD510258CE510358CF51045804E201EB64
:105D00009DF202EB9EF2ABDFCBD8D890F45004E6C4
:105D1000800ECC5D0C0ECD5907E201EB9DF202EB3B
:105D20009EF20201A1693BD0043401E2C9D8640E9D
:105D3000D06FD16BD26BD36B9DC2D8F19EC2D9F11B
:105D4000DA6BDB6BD9AF02D0DA69DB69D8C1E6FF69
:105D5000D9C1E6FFDAC1E6FFDBC1E6FFE66EE66A1F
:105D6000E66AE66ABBD8DCEC2CF023EC2CF0E552BA
:105D7000E5CFD7F1E5CFD6F1E5CFD5F1E7CFD4F137
:105D80000101D451D05DCC6FD551D159CD6FD651D1
:105D9000D259CE6FD751D359CF6FCCC1A1F28CD08D
:105DA0005ED882E941E8E66A30EC2AF041E9E66A29
:105DB00018EC2BF041E9005008E0E66ABCEC3CF03E
:105DC00041E9E66ABCEC3CF041E95AD821E0020125
:105DD0009F519D1902E1A0519E1901E045D84FDF66
:105DE0005FD8F43406E2CC510008000ECD5501E234
:105DF0005DD8E668AA0EE66EF2EC1DF042E936ECDC
:105E00003EF093909392080E8A6E816ED190FFD7E8
:105E1000E66830EC2AF041E93F0EE66E18EC2BF014
:105E200041E942E9E7CFD9FF120058D8DDEC34F060
:105E300048E9A2C2CCF1A3C2CDF1A4C2CEF1A5C261
:105E4000CFF1010142D803EBF3FF04EBF4FF1200A2
:105E5000E66E680EE66EB2EC3AF043E91200D9CF76
:105E6000E6FFE1CFD9FF1200020EE66E9D0EE66E50
:105E7000020EE66EF20EE66E27EC1EF044E912000A
:105E8000080EE66E680EE66E67EC3AF042E9F350F3
:105E9000800B12002CD8F350036EF450046E1200E5
:105EA000F3CFCCF1F4CFCDF101011200000EE66E7C
:105EB000E66AE8DE42E9120045E9E7CFD9FF1200C1
:105EC000016A026A036A046A1200CC51016ECD5164
:105ED000026ECE51036ECF51046E120001EBE6FF4D
:105EE00002EBE6FF03EBE6FF04EBE6FF1200E66ED3
:065EF0005CDE41E9120036
:0A5EF6006C5007E1689667D902E1DD
:105F00000AD8010C37D8010C040E6C5C03E16896CA
:105F100040D8010C000C54D941E8040104BF046BC3
:105F200002019C6B946B956B9A6B9B6B60EC32F0EF
:105F3000016A010E52D919E20201955116E1F76A80
:105F40000134FE0BF66EF736EC0EF626720EF722D3
:105F50000900F5CFCCF10800F5CFCDF1CDC1FAFFA6
:105F60000101CC511400012AE4D7A3D842E9E7CFBC
:105F7000D9FF1200020E0201945D09E170D80401FC
:105F800000BD02D0C80E01D0880E006F120092EF43
:105F900030F0040E0201A65D09E122C46EFF6E50CE
:105FA000000802E2050E01D0030EA66F020194055F
:105FB00010E111D8020E02019C5D03E10401840E80
:105FC00006D0040104BD02D0C80E01D0880E046FB3
:105FD000120092EF30F0F4D842E80201200E9A5DF0
:105FE000000E9B590DE29A51016E9B51026E9C511D
:105FF00002E1010E03D09C0506E1020E9C6F03D066
:10600000200E016E026A04010493049102500413ED
:1060100001EB05F4015002019A5F02509B5B400EB8
:10602000986F040E996F0201A7A30BD001500210C4
:1060300012E096C2F6FF97C2F7FF0800F550B0D8FD
:10604000F5D70150021007E096C2E9FF97C2EAFFB8
:10605000EF50A6D8F6D743E9E7CFD9FF1200B0D862
:1060600042E8030E04010015026E0151016E9A0E02
:10607000E96E020EEA6E0201EE5001249A6FED50B5
:1060800002209B6F400E966F040E976F0150021016
:106090000CE096C2E9FF97C2EAFFEF5098C2E9FF11
:1060A00099C2EAFFEF6EA0D8F1D743E9E7CFD9FF55
:1060B00012006D980201955105E17AD8840E006FA7
:1060C00004011DD0040120AF1CD002019A5104012B
:1060D000265D02019B510401275904E226C49AF26D
:1060E00027C49BF278DF0201010E946F61D8800E05
:1060F000006F0401400E066F040E076FC80E046F98
:1061000012000201020E946F0401056BC80E046FA9
:106110000401200E016F400E026F040E036FC80EC3
:10612000006F12004DD841E8020E0201945D2DE18E
:106130006D50100B2AE0040101510101CC6FCD6BB1
:10614000200ECC1922E1CD5120E140D81EE10051B2
:10615000800B1BE1200E026F040E036F016A200EFC
:106160003CD81AE20150EA6A400FE96E040EEA22B6
:10617000EF50E66E0150EA6A200FE96E040EEA2243
:10618000E552E750EF6E012AEAD70201946B10D86E
:106190008C0E006F0401046B42E9E7CFD9FF1200B7
:1061A00098C2E9FF99C2EAFFEF6E0201F4EF30F006
:1061B0000401200E016F200E026F040E036F120007
:1061C000D9CFE6FFE1CFD9FF81E9120004010051E8
:1061D0003C0BE842E8420D081200F36EF46AF350FB
:1061E000015C000EF4541200982B000E9923962B9C
:0861F00097230106025A120078
:0861F800040120511F0B0108F6
:1062000001E012002051600BE842E842E842E84217
:10621000E842010801E01200245103E0240501E0F6
:1062200012002151230A39E0010A33E0030A25E074
:10623000010A1CE0240A31E0070A2FE0010A2DE0E0
:10624000030A0EE0010A01E0120031D90201F20E48
:10625000966F000E976F0201A7930201080E17D0E8
:1062600026D90201F20E986F000E05D020D9020146
:10627000EA0E986F000E996F120019D90201EA0E0A
:10628000966F000E976F0201A7930201070E9A6F97
:1062900012000DD922C4F1F0120012000001EA6BC5
:1062A000C20EEB6F010EEC6FED6BEE6BEF6B080E39
:1062B000F06FE36BE26B1A0E726E1E0E736E0401CA
:1062C000600E166F040E176F400E146F0401196FE5
:1062D000680E1A6F040E1B6F880E186F0401A80E4B
:1062E0001E6F040E1F6F400E1C6F1200E4D884E96D
:1062F0000001E26B040118BF24D00050195D02E2D6
:106300001951006E0001E26B0050E25D13E2E251B0
:10631000EA6A680FE96E040EEA22EF50E66EE25177
:106320000124E96E000E0220EA6EE552E750EF6E9E
:10633000E22BEAD70401400E196F1817187D880E5A
:1063400018130001E25141E9E7CFD9FF12009ED8AE
:1063500012E1036AA1D802E1F45009E000EBE9FF81
:1063600001EBEAFF002A000E0122EF50F3E176D89C
:10637000E96B010EE36F97D089D813E1036A8CD8DB
:1063800002E1F4500AE000EBF6FF01EBF7FF002A10
:10639000000E01220800F550F2E160D8010EE96F0D
:1063A000E36F81D088D881E941E804011CBF55D052
:1063B000030E0001E35D01E1E36BE3514EE0020EE9
:1063C000E35D03E104011D6B3FD0E30540E1E851CB
:1063D0000101CC6FCD6BCC514008000ECD5502E2CF
:1063E000400E02D00001E851016E01EB1DF4015096
:1063F0000001E85DE86FA80EE66F040EE76FE9059F
:106400000AE1015011E0E4C0F6FFE5C0F7FF080023
:10641000F55030D8F6D7015007E0E4C0E9FFE5C0F9
:10642000EAFFEF5027D8F7D70001E85110E1040147
:106430001D510101CC6FCD6B400ECC1905E1CD5142
:1064400003E10001020E02D00001030EE36F400ED3
:1064500004011C171C7D880E1C1325D00350005E00
:10646000000E015A00EBE4F001EBE5F003EBE8F07D
:1064700000011200E6C0E9FFE7C0EAFFEF6EE62B7D
:10648000000EE723E42BE5230106120014D883E96C
:1064900041E80001E3511200032AFF0EF36EF46A93
:1064A000F3500318120042E9E7CFD9FF12000201AE
:1064B000030E956F1200D9CFE6FFE1CFD9FF12008E
:1064C00004012051600BE842E842E842E842E84219
:1064D000000901E012002151070A3FE00B0A3DE0EC
:1064E000070A32E0010A23E00B0A1FE0020A1DE05E
:1064F000030A19E0080A10E0010A0CE00F0A08E09C
:10650000030A01E0120015D90201040EA66F120061
:10651000AEEF32F0E5EF32F00CD90201A80E966F23
:10652000020E976F0BD006EF33F038EF33F005D93A
:106530000201976BA90F966F020E97230201A79392
:106540000201010E9A6F1200F8D8EA6AA90FE96EEB
:10655000020EEA2222C4EFFF12001200800E040194
:10656000205D32E12351030A1FE0010A0AE0030A19
:1065700029E1DFD80201210E966F720E976F120E7D
:106580001ED0C6D8E20EF626720ECBD8020E02013D
:10659000F76A9625F66E9751F7220900F5CF9AF221
:1065A0000A00F5CF9BF20ED0B3D8E60EF626720E97
:1065B000B8D896C2F6FF97C2F7FF0800F55002015F
:1065C0009A6F9B6B0201A7831200B3D80F0EE66E81
:1065D000710EE66E0F0EE66ED1EC37F043E9010E58
:1065E000E66EA90EE66E020EE66ED1EC37F043E9D8
:1065F00022C4A8F20401225104E10201050EA66F93
:1066000012000201060EA66F4EEF31F00401406B3E
:10661000416B040120511F0B020A0FE0030A0BE03B
:10662000010A18E186D8040140810201A7A112D015
:10663000040140830FD07DD80DD050D801E0010E69
:106640005BD898C2E9FFEA6EEF50040B03E0040147
:10665000010E406F020195050AE10201400E966F9E
:10666000040E976F0201A7930201020E9A6F1200A7
:10667000040122050EE120511F0B00090AE159D83F
:10668000030E0401215D03E10201A78102D0020192
:10669000A7910401225121E120511F0B02081DE1A5
:1066A00024510F0B000919E019D801E0010E24D87C
:1066B000030E0401215D02E1840E03D024AF07D054
:1066C000400E98C2E9FF99C2EAFFEF6E1200880EF1
:1066D00098C2E9FF99C2EAFFEF6E12002ED80F0BA5
:1066E000080DF3500101CD6B000FCC6F040ECD23CC
:1066F00004012451800B1200040DF3500101CC253C
:106700000201986F000E0101CD210201996F120064
:1067100010D804012251F66EF76AD890F636F73693
:106720001200F7220900F5CF96F20A00F5CF97F292
:1067300012000201010E956F1200FBDF04012451CB
:02674000120045
:0E674200D9CFE6FFDACFE6FFFA0EE3CFD9FF9C
:10675000FB0EE3CFDAFFFC0EE3CFE9FFFD0EE3CF44
:10676000EAFFE9CFF3FFEACFF4FFF80EE35003E1CD
:10677000F90EE35008E0F80EE30602E2F90EE30634
:10678000DECFEEFFF2D7FF0EE3CFDAFFE552FF0ECA
:10679000E3CFD9FFE5521200FB0EE3CFF6FFFC0E6C
:1067A000E3CFF7FFFD0EE3CFF8FFFE0EE3CFE9FFE7
:1067B000FF0EE3CFEAFFE9CFF3FFEACFF4FFF90ED4
:1067C000E35003E1FA0EE35009E0F90EE30602E2BA
:1067D000FA0EE3060900F5CFEEFFF1D71200FE0E28
:1067E000E3CFE9FFFF0EE3CFEAFFE9CFF3FFEACF04
:1067F000F4FFFB0EE35003E1FC0EE35009E0FB0E57
:10680000E30602E2FC0EE306FD0EE350EE6EF1D766
:106810001200D9CFE6FFDACFE6FFFA0EE3CFD9FFB9
:10682000FB0EE3CFDAFFFC0EE3CFE9FFFD0EE3CF73
:10683000EAFFE9CFF3FFEACFF4FFEE66FED7ED52B1
:10684000DFCFEEFFDE66FCD7FF0EE3CFDAFFE552C7
:10685000FF0EE3CFD9FFE5521200FB0EE3CFF6FFA8
:10686000FC0EE3CFF7FFFD0EE3CFF8FFFE0EE3CF04
:10687000E9FFFF0EE3CFEAFFE9CFF3FFEACFF4FF32
:10688000EE66FED7ED520900F5CFEFFFEE66FBD7BF
:106890001200FE0EE3CFE9FFFF0EE3CFEAFFFD0E8D
:1068A000E350EF5C05E0EE66FAD7F36AF46A04D0D1
:1068B000E9CFF3FFEACFF4FF1200FB0EE3CFF6FFC0
:1068C000FC0EE3CFF7FFFD0EE3CFF8FFFE0EE3CFA4
:1068D000E9FFFF0EE3CFEAFFE9CFF3FFEACFF4FFD2
:1068E0000900F5CFEFFFEE66FBD71200FE0EE3CFF7
:1068F000E9FFFF0EE3CFEAFFF36AF46AEE5203E02A
:10690000F34AF42AFBD71200D9CFE6FFDACFE6FF2D
:10691000FA0EE3CFD9FFFB0EE3CFDAFFFC0EE3CF95
:10692000E9FFFD0EE3CFEAFFF80EE35003E1F90EB5
:10693000E3500AE0F80EE30602E2F90EE306DE5049
:10694000EF5C02E1EE66F0D7F36EFF0EE3CFDAFF05
:10695000E552FF0EE3CFD9FFE552F3501200D9CF35
:10696000E6FFDACFE6FFFA0EE3CFD9FFFB0EE3CF67
:10697000DAFFFC0EE3CFE9FFFD0EE3CFEAFFE9CF3C
:10698000F3FFEACFF4FFF80EE35003E1F90EE35012
:106990000BE0F80EE30602E2F90EE306DECFEFFFAE
:1069A000EE66F1D7DD52EFD7FF0EE3CFDAFFE55207
:0A69B000FF0EE3CFD9FFE5521200FD
:0669BA000BD8E552E5CF09
:1069C000A5F2E5CFA4F2E5CFA3F2E7CFA2F248E823
:1069D000000C46E8D9CFE6FFDACFE6FFE1CFD9FFDA
:1069E000E2CFDAFF90E90A6A0B6A0C6A0D6A00507E
:1069F0000502F450086E01500402F4500826000EFF
:106A0000096A092200500602F3500826F4500922B0
:106A1000000E0A2201500502F3500826F450092204
:106A2000000E0A2202500402F3500826F4500922F4
:106A3000000E0A2200500702F3500926F4500A22E1
:106A4000000E0B2201500602F3500926F4500A22D0
:106A5000000E0B2202500502F3500926F4500A22C0
:106A6000000E0B2203500402F3500926F4500A22B0
:106A7000000E0B2201500702F3500A26F4500B229D
:106A8000000E0C2202500602F3500A26F4500B228C
:106A9000000E0C2203500502F3500A26F4500B227C
:106AA000000E0C2202500702F3500B26F4500C2269
:106AB000000E0D2203500602F3500B26F4500C2258
:106AC000000E0D2203500702F3500C26F4500D2245
:106AD000000E0E2207AE06D000500A5E01500B5A7F
:106AE00002500C5A03AE06D004500A5E05500B5AF1
:106AF00006500C5A89EB00F08AEB01F08BEB02F0A8
:106B00008CEB03F0E552E5CFDAFFE7CFD9FF4AE996
:106B1000000C0AD844E9E6CFA2F2E6CFA3F2E6CF12
:106B2000A4F2E6CFA5F2000C46E8D9CFE6FFDACF13
:106B3000E6FFE1CFD9FFE2CFDAFF8CE944E8036654
:106B400024D082EB09F0010E0F6E200E0E6E0D6A3E
:106B50000C6A010E076E800E066E056A046A040E4A
:106B6000086E09361FE2093609E384EB0CF085EB69
:106B70000DF086EB0EF087EB0FF014D0D8900E36A8
:106B80000F3606360736082EECD7660E83EB09F073
:106B9000094ECD0E094EA60E094E880E0E6E0C6AD9
:106BA0000D6A0F6A080E0201B567B551086E0CEB4D
:106BB000E6FF0DEBE6FF0EEBE6FF0FEBE6FF00EB6B
:106BC000E6FF01EBE6FF02EBE6FF03EBE6FF0CEB73
:106BD000E6FF0DEBE6FF0EEBE6FF0FEBE6FFE9EC61
:106BE00034F0E9EC34F0000ED880105611561256ED
:106BF000030E1356E9EC34F0D8900F320E320D32FA
:106C00000C32082ED4D7E552E550036EE550026EE3
:106C1000E550016EE750006EE552E5CFDAFFE7CFB1
:066C2000D9FF46E9000C5B
:0A6C2600ECD883E901340AE300EB27
:106C3000CCF101EBCDF10101CC6DCD1F000ECD23C8
:106C400004D000EBCCF101EBCDF1CCC1F3FFCDC111
:106C5000F4FF41E9E7CFD9FF1200D2D886E949E82D
:106C6000C9D800EBE6FF01EBE6FFE3EC37F044E9BF
:106C7000C1D876EC34F042E9F3500E6E0E50025C4F
:106C80000E6E0E3401E30E6A0E50025C0101CC6FF1
:106C9000CD6B800B01E0CD69CCC1E6FFCDC1E6FF35
:106CA000A9D80EEBD0F1D16BD0BFD1690350D0255C
:106CB000CE6F0450D121CF6FCEC1E6FFE66EA1ECBE
:106CC00033F046E94AE9E7CFD9FF120099D886E9BF
:106CD000013402E32D0E01D02B0EE66E03EBE9FF2B
:106CE00004EBEAFFE552E750EF6E00EBE6FF01EB45
:106CF000E6FF99DF42E9F3CFE6FFF4CFE6FF02EBD0
:106D0000E6FF03EBE6FF04EBE6FFA7DF45E941E919
:106D1000E7CFD9FF120074D887E941E8076A033446
:106D20000350071802E60350075C36E203EBD0F18C
:106D30000101D16BD0BFD1693FD8D2BFD36965D82B
:106D4000EF380F0BF66EF76AF6BEF76849D8CC6FCE
:106D5000CD6B800B01E0CD693CD8E552E750EF6E7A
:106D600003EBD0F1D16BD0BFD16926D8D2BFD369A4
:106D70004CD8EF500F0BF66EF76AF6BEF76830D8B6
:106D8000010FCC6FCD6B800B01E0CD6922D8E552AD
:106D9000E750EF6E072AC3D700500AE00750E824F7
:106DA0000101CC6FCD6B800B01E0CD6912D8EF6A89
:106DB00042E9E7CFD9FF12000150D025CE6F025033
:106DC000D121CF6FCE07000ECF5B07EBD2F1D36B93
:106DD0001200CC510424E96ECD510520EA6E120058
:106DE000020EF6267C0EF7220800F550E66E0750DC
:106DF000E8241200D950060FE66EDACFE6FF120043
:106E0000D9CFE6FFE1CFD9FF1200D251CE5DE96EB6
:086E1000CF51D355EA6E1200C8
:086E180081B804D06DB604D06E
:106E20000FD802D06DB613D80201A60508E16DBADD
:106E300006D0686A696A69806988020EA66F1200C6
:106E40006D6A696A6D860201010EA66F12006D6A95
:106E5000696A0201A66B120027EF37F00201A65102
:106E600001E112006850040B04E06950040B01E0DA
:106E700045D86DB212006850010B04E06950010B57
:106E800001E069D86850100B04E06950100B01E074
:106E90002ED86850400B04E06950400B01E047D801
:106EA0006850200B04E06950200B01E042D8685084
:106EB000020B04E06950020B01E04BD8030E020103
:106EC000A65D01E212000201AE6B040EAE5D0EE2A1
:106ED0006850080B0BE06950080B08E07BEC2FF0C2
:106EE000000901E168960201AE2BEFD71200698418
:106EF00068986D82A19AA08AA09A12006D926994F6
:106F000068A402D06894FCD712000201A7A10ED099
:106F10006D926D840201080EAF6F070EB06FAF0760
:106F2000000EB05BAF51B011FAE16D941200689C95
:106F3000120070A00CD0800E0401005D07E1840EE9
:106F40000401045D03E104018C0E006F7090689AE7
:106F500012006A6A12006A6A686A9F0E6B6E7B0E84
:106F6000696E6E6A0F0EE66E710EE66E0F0EE66EBD
:106F700018D843E9160E706E68A608D0689600000F
:106F800000000000000000000000F6D76D9892ECB1
:106F900030F00201A7910201A86B0201030EA66F57
:106FA0001200D9CFE6FFE1CFD9FF84E901EBE9FF79
:106FB00002EBEAFF005003E0EE6A0006FBD741E96E
:066FC000E7CFD9FF12002B
:0A6FC600D9CFE6FFDACFE6FFFA0E9E
:106FD000E3CFD9FFFB0EE3CFDAFFFD0EE35209E763
:106FE0002D0EDE6EFC0EE31EE32AFD0ED8B4E30682
:106FF000E31EE652E652E652FD0EE124E76EFF0E76
:10700000E220E46EE652F70EE3CFE6FFF70EE3CFA1
:10701000E6FF53EC38F0F90EE124E96EFF0EE220B2
:10702000EA6E43EC38F00AE140EC38F009E143EC59
:1070300038F008E140EC38F007E108D04EEC38F0C9
:1070400049EC38F04EEC38F049EC38F04EEC38F0C2
:10705000DE6AF90EE126FF0EE222FF0EE3CFDAFF31
:10706000E552FF0EE3CFD9FFE552FC0EE124E96EB5
:10707000FF0EE220EA6EEECFF3FFEFCFF4FF120037
:10708000EF380F0B1200EF500F0B02E1EE52D884D5
:107090001200EF380F0B300FDE6E1200EE500F0BA8
:1070A000300FDE6E1200FC0EE3CFE9FFFD0EE3CFE2
:1070B000EAFF100EE66EEE6AEE6AEF6AD890FD0EF9
:1070C000E336FE0EE336ED36ED36EF36FF0EE30621
:1070D00009E074EC38F0EE5274EC38F0EE5274ECD7
:1070E00038F0EDD7E56E1200030EEF24E8B6EF6E30
:0A70F000300EEF24E8BEEF6E000C36
:0670FA0000000000000090
:107100005F00000000030003000006090906242AAE
:107110007F2A1223130864623649562050000B0759
:10712000000000003E410000413E0000082A1C2AE9
:107130000808083E08080058380000080808080831
:10714000003030000020100804023E5149453E0046
:10715000427F40006251494946224149493618144C
:10716000127F1027454545393C4A4949300171098C
:1071700005033649494936064949291E0036360075
:1071800000005B3B00000008142241141414141486
:10719000412214080002015109063E415D551E7E40
:1071A0000909097E7E494949363E414141227F41D4
:1071B00041413E7F494949417F090909013E414119
:1071C00051327F0808087F00417F41002040404045
:1071D0003F7F081422417F404040407F020C027FE5
:1071E0007F0408107F3E4141413E7F090909063E68
:1071F0004151215E7F091929462649494932010139
:107200007F01013F4040403F07186018077F20186A
:10721000207F631408146303047804036151494513
:01722000432A
:0F7221001201000202000020D8040A0000000140
:10723000020001090243000201008032090400003B
:1072400001020201000524001001042402020524A9
:107250000600010524010001070582030800020958
:10726000040100020A0000000705030240000007B5
:1072700005830240000004030904340355006E0036
:1072800064006500720077006F006F0064002000EA
:1072900055006E00640065007200670072006F00A8
:1072A00075006E00640020002000200020003403E0
:1072B00053006800650074006C0061006E0064009B
:1072C0002000410074007400610063006B00200026
:1072D00050006F006E007900200020002000200088
:0E72E00020003372337276727A72AE72F861E9
:0272EE0030303E
:1072F00030302030303030003030303300303030FB
:10730000203030300058585858585858582058583D
:10731000585858585858205858585858585858007D
:1073200048697961004552585800434C5858004C00
:10733000303030004D30303000484F4C4400534125
:10734000564500524157200048494748004752419E
:10735000440043414C200020303023005341502052
:1073600000303030250048454C500030303030007F
:107370003030304700433030300030303023002A86
:1073800020200D0A0024505450534854442C0030FF
:0673900030303030300007
:0A7396002A0EF66E080EF76E000EC8
:1073A000F86E02010900F5508F6F0900F550906FDB
:1073B00003E18F6701D03DD00900F5508A6F0900C5
:1073C000F5508B6F0900F5508C6F09000900F550DE
:1073D000E96E0900F550EA6E090009000900F55050
:1073E0008D6F0900F5508E6F09000900F6CF91F2FC
:1073F000F7CF92F2F8CF93F28AC2F6FF8BC2F7FF73
:107400008CC2F8FF02018D5302E18E5307E00900A0
:10741000F550EE6E8D07F8E28E07F9D791C2F6FFB0
:1074200092C2F7FF93C2F8FF02018F07000E905B34
:04743000BFD71200B0
:0C743400D9CFE6FFDACFE6FFE1CFD9FFA9
:10744000E2CFDAFF87E911EC3EF0C580C5B0FED788
:10745000A1B62CD004EBE6FF35D80FE1C5BC28D08F
:1074600003EBE6FF2FD809E1C5BC22D0C582C5B227
:10747000FED70428E66E26D803E0C584FD0E1CD096
:10748000C5BC16D000EBE6FF01EBE6FF02EBE6FF22
:10749000DFEC3BF043E9000909E1C58AC588C5B8BE
:1074A000FED7C584C5B4FED7A1A605D0FF0E04D073
:1074B000C584FE0E01D0000E41E9E5CFDAFFE7CF2B
:0E74C000D9FF120033EC3CF041E90009120044
:0274CE00D9CF14
:1074D000E6FFDACFE6FFE1CFD9FFE2CFDAFF84E9BA
:1074E00011EC3EF0C580C5B0FED7A1B626D001EBA9
:1074F000E6FF33D811E1C5BC22D000EBE6FF2DD862
:107500000BE1C5BC1CD0C582C5B2FED7A1B615D053
:107510000128E66E22D803E0C584FD0E12D0C5BC5A
:107520000ED0C586C5B6FED7C58AC588C5B8FED7F4
:10753000C584C5B4FED7A1A607D0F36803D0C5841F
:10754000FE0EF36EF46803D0C950F36EF46A41E99D
:10755000E5CFDAFFE7CFD9FF120033EC3CF041E989
:04756000000912000C
:0C756400D9CFE6FFDACFE6FFE1CFD9FF78
:10757000E2CFDAFF85E911EC3EF0C580C5B0FED759
:10758000A1B61BD002EBE6FF21D80CE1C5BC0DD0A3
:1075900001EBE6FF1BD806E1C5BC07D000EBE6FF18
:1075A00015D806E0C584FD0E0BD0C584FE0E08D0AC
:1075B000C584C5B4FED7A1A602D0FF0E01D0000E2F
:1075C00041E9E5CFDAFFE7CFD9FF120033EC3CF019
:0675D00041E90009120070
:0A75D60000000000000000000000AB
:1075E000000000000000000000000000000000009B
:1075F000000000000000000000000000000000008B
:10760000000000000000000000000000000000007A
:10761000000000000000000000000000000000006A
:10762000000000000000000000000000000000005A
:0E76300000000000000000000000000000004C
:02763E00F36AED
:10764000F46AFF0EE124E96EFF0EE220EA6EED66B9
:1076500013D02F0EEF6410D0390EEF640CD0400E13
:10766000EF640AD05A0EEF6406D0600EEF6404D0C7
:107670007B0EEF6001D0F32A1200F36AF46AFF0E6A
:10768000E124E96EFF0EE220EA6EED660AD0200EDC
:10769000EF5C06E0080EEF6404D00E0EEF6001D040
:0476A000F32A1200B7
:0C76A400D9CFE6FFE1CFD9FF82E941E831
:1076B000080E026E00EBB2F28B940201B2BF8B8413
:1076C00000000000D8908BB4D8808B90B2370000B7
:1076D00000000000000000000000000000000000AA
:1076E000000000008B808B940201B2BF8B840206E5
:1076F0000250E8E10201B25100D042E9E7CFD9FFE0
:02770000120075
:0E770200D9CFE6FFDACFE6FFE1CFD9FFE2CF25
:10771000DAFF83E944E8F8CF05F0F6CF06F00C0E67
:10772000BA6E050EF66EF76A300EF86E0800F55068
:10773000010B02E0046801D0046A045002E0949254
:1077400001D09396CA9400EBCBFFCA8405C0F8FF22
:1077500006C0F6FF45E9E5CFDAFFE7CFD9FF120013
:10776000D9CFE6FFDACFE6FFE1CFD9FFE2CFDAFFEC
:1077700085E9C26AC06A01407F0B3C0BC26E0138CA
:10778000F00B300B0010C16E0250040DF350380B9B
:107790000101CD6F02380F0B070BCC6F800E021466
:1077A000CC11CD11C06E01AE03D09E9C9D8CF28C8D
:0E77B000C28041E9E5CFDAFFE7CFD9FF120032
:0277BE00D9CF21
:1077C000E6FFDACFE6FFE1CFD9FFE2CFDAFF85E9C6
:1077D0000050000600091AE024EC3EF0E66E01EBD2
:1077E000E9FF02EBEAFF012A000E0222E552E75010
:1077F000EF6EC5B6FED7A1A602D0FF0E08D000508E
:10780000E7E0C59AC588C5A8E3D7FDD7000E41E9D2
:0A781000E5CFDAFFE7CFD9FF120041
:06781A00D9CFE6FFDACF32
:10782000E6FFE1CFD9FFE2CFDAFF84E942E880EB5F
:1078300004F081EB05F0060ED89004360536E80416
:10784000FBE105EBBBFF0440E8423F0B300B0101BD
:10785000CC6FCF0EBA14CC11BA6E43E9E5CFDAFF84
:06786000E7CFD9FF120082
:0A786600D9CFE6FFDACFE6FFE1CF4D
:10787000D9FFE2CFDAFF83E900EBC9FFC6AE02D041
:10788000FF0E11D0C7B0FED70F0EC614080804E0D3
:107890000F0EC614090802E111EC3EF0C5AC02D08F
:1078A000FE0E01D0000E41E9E5CFDAFFE7CFD9FFA8
:0278B0001200C4
:0E78B200D9CFE6FFDACFE6FFE1CFD9FFE2CF74
:1078C000DAFF84E9ACA2FED700EBE9FF01EBEAFFA7
:1078D000EFCFE6FFB6EC3DF041E900EBE9FF01EB4D
:1078E000EAFF002A000E0122EF50ECE141E9E5CF6A
:0878F000DAFFE7CFD9FF120017
:0878F800D9CFE6FFDACFE6FF6D
:10790000E1CFD9FFE2CFDAFF83E9360E0014B16E82
:10791000B36AB26AA19200AE02D0A08201D0A09256
:1079200000A002D0B18E01D0B19EB18041E9E5CF77
:08793000DAFFE7CFD9FF1200D6
:08793800D9CFE6FFDACFE6FF2C
:10794000E1CFD9FFE2CFDAFF83E97E0E0014CD6EDE
:1079500000AC02D0CD8E01D0CD9ECF6ACE6A9E9073
:1079600000AE02D09D8001D09D90CD8041E9E5CF51
:08797000DAFFE7CFD9FF120096
:08797800FF0EE3500201B16FA4
:10798000EE0E02D0F20E0000E76EE72EC5EF3CF0DF
:107990000C0E0101FF6FE76AE72ECCEF3CF0FF2FE2
:0E79A000CBEF3CF00201B12FC2EF3CF0120021
:0279AE00D9CF2F
:1079B000E6FFDACFE6FFE1CFD9FFE2CFDAFF83E9D6
:1079C0007F0E0014D56ED76AD66AF29400AE02D04C
:1079D000F28A01D0F29AD58E41E9E5CFDAFFE7CFFE
:0479E000D9FF1200B9
:0C79E400D9CFE6FFDACFE6FFE1CFD9FFF4
:1079F000E2CFDAFF83E9FB0E0014CA6ECC6A9E92D6
:107A000000AE02D09D8201D09D92CA8441E9E5CFAB
:087A1000DAFFE7CFD9FF1200F5
:087A1800D9CFE6FFDACFE6FF4B
:107A2000E1CFD9FFE2CFDAFF84E93F0EC716C66A7D
:107A3000C56A0150C6120050C71293829380C68A4D
:0C7A400041E9E5CFDAFFE7CFD9FF1200E3
:047A4C00D9CFE6FFA9
:107A5000DACFE6FFE1CFD9FFE2CFDAFF84E942E8EF
:107A600080EB04F081EB05F005EBB3FF04EBB2FF14
:0C7A700043E9E5CFDAFFE7CFD9FF1200B1
:047A7C00D9CFE6FF79
:107A8000DACFE6FFE1CFD9FFE2CFDAFF82E942E8C1
:107A9000B250026EB350036E02EBF3FF03EBF4FF40
:0C7AA00043E9E5CFDAFFE7CFD9FF120081
:047AAC00D9CFE6FF49
:107AB000DACFE6FFE1CFD9FFE2CFDAFF84E942E88F
:107AC00080EB04F081EB05F005EBCFFF04EBCEFF7C
:0C7AD00043E9E5CFDAFFE7CFD9FF120051
:047ADC00D9CFE6FF19
:107AE000DACFE6FFE1CFD9FFE2CFDAFF82E942E861
:107AF000CE50026ECF50036E02EBF3FF03EBF4FFA8
:0C7B000043E9E5CFDAFFE7CFD9FF120020
:047B0C00D9CFE6FFE8
:107B1000DACFE6FFE1CFD9FFE2CFDAFF84E942E82E
:107B200080EB04F081EB05F005EBD7FF04EBD6FF0B
:0C7B300043E9E5CFDAFFE7CFD9FF1200F0
:047B3C00D9CFE6FFB8
:107B4000DACFE6FFE1CFD9FFE2CFDAFF82E942E800
:107B5000D650026ED750036E02EBF3FF03EBF4FF37
:0C7B600043E9E5CFDAFFE7CFD9FF1200C0
:047B6C00D9CFE6FF88
:107B7000DACFE6FFE1CFD9FFE2CFDAFF83E9ACACA1
:107B800004D0AC900201B3B3AC8000EBADFF41E98F
:0A7B9000E5CFDAFFE7CFD9FF1200BE
:067B9A00FF0EE3500201A2
:107BA000B16F1A0E00D000D001D0200EE76EE72E84
:0A7BB000FED7B12FFAD700D0120063
:067BBA0013EE00F023EEC3
:107BC00000F0F86ACBEC39F03CEC3EF0CFEC04F07E
:047BD000FBD71200CD
:0C7BD400C4CFCEF1CEC1CFF10101CE6BC9
:0C7BE000C350CE11F36ECFC1F4FF1200B1
:047BEC00FF0EE35055
:107BF000E84E1200000000D000D000D0E82EFAD7E6
:027C0000120070
:0E7C020030313233343536373839414243445D
:037C1000454600E6
:017C13000070
:0C7C14008B8E8B948B80949E94949490A3
:027C2000120050
:0E7C22001F0EC514FDE1C750040BFAE112005D
:0E7C300000EE00F00F0EEE6AEA62FDD71200C1
:027C3E000A4FEB
:087C40004B0A000A4B4F0A0039
:087C4800C586C7A0FED7C95094
:027C5000120020
:0A7C5200C250020B01E0010E120007
:047C5C00B190A092B1
:027C6000120010
:067C6200C2909D9C12007F
:047C68008B8E1200ED
:047C6C00C69A1200A2
:047C70008B9E1200D5
:047C7400C2821200B6
:027C78001200F8
:047C7A003D0A270098
:027C7E00C771CC
:0B7C80001C010000000A0000010000D1
:057C8B000101FFFF01F3
:017C900001F2
:017C910003EF
:0C7C9200B84B390049920400000040008B
:020000040030CA
:0100000038C7
:010001000EF0
:010002001CE1
:010003001CE0
:01000500807A
:01000600C138
:010008000FE8
:01000900C036
:01000A000FE6
:01000B00E014
:01000C000FE4
:01000D0040B2
:0200000400F00A
:0100FF00AA56
:00000001FF
